:100000000C9478090C9499090C9499090C94990909
:100010000C9499090C9499090C9499090C949909D8
:100020000C9499090C9499090C9499090C949909C8
:100030000C9499090C9499090C9499090C949909B8
:100040000C9499090C94AC140C9499090C9499098A
:100050000C9499090C9499090C94C3120C94C54CF6
:100060000C9499090C9480490C9499090C94990961
:100070000C9499090C9499090C9499090C94990978
:100080000C9499090C9499090C9499090C94990968
:100090000C9499090C9499090C9499090C94990958
:1000A0000C9499090C9499090C9499090C94990948
:1000B0000C9499090C9499090C9499090C94990938
:1000C0000C9499090C9499090C9499090C94990928
:1000D0000C9499090C9499090C9499090C94990918
:1000E0000C949909151321133D13491363136F13CE
:1000F00089138B13D84DDB4DCE4DD24D124EDF4DB3
:10010000E34DE94DED4DF14DF74DFB4DFF4D124ED9
:10011000054E094E0D4ECC4ED14ED64EE04E594FA7
:10012000EA4EF24EFA4E044F0E4F184F274F314F02
:10013000594F3B4F454F4F4F084AD73B3BCE016E7F
:1001400084BCBFFDC12F3D6C74319ABD56833DDA2E
:100150003D00C77F11BED9E4BB4C3E916BAAAABE3D
:10016000000000803F05A84CCDB2D44EB93836A966
:10017000020C50B9918688083CA6AAAA2ABE0000A3
:1001800000803F54656D706572617475726520689A
:10019000656174656420626564207377697463685F
:1001A0006564206F66662E204D415854454D5020A1
:1001B000747269676765726564202121003A204581
:1001C00078747275646572207377697463686564A6
:1001D000206F66662E204D494E54454D5020747256
:1001E000696767657265642021003A2045787472FA
:1001F00075646572207377697463686564206F66DF
:10020000662E204D415854454D50207472696767E1
:1002100065726564202100202D20496E76616C692D
:1002200064206578747275646572206E756D6265A0
:1002300072202100504944204175746F74756E65B9
:100240002066696E6973686564202120506C616363
:100250006520746865204B702C204B6920616E64AA
:10026000204B6420636F6E7374616E747320696ECB
:100270002074686520636F6E666967757261746962
:100280006F6E2E6800504944204175746F74756E0E
:1002900065206661696C6564212074696D656F75A0
:1002A000740020403A006F6B20543A006F6B20427C
:1002B0003A00504944204175746F74756E6520662C
:1002C00061696C6564212054656D70657261747537
:1002D000726520746F206869676800204B643A205B
:1002E00000204B693A2000204B703A200020436CDC
:1002F000617369632050494420002054753A2000FE
:10030000204B753A2000206D61783A2000206D69FD
:100310006E3A200020643A200020626961733A201E
:10032000004572726F723A001000F401E0020E0193
:100330002003090160030401A003FF00E003FA00A9
:100340003004F5008004F000F004EB005005E600F6
:10035000B005E1003006DC00B006D7004007D2004F
:10036000E007CD008008C8005009C300000ABE00A5
:10037000F00AB900F00BB400100DAF00000EAA0097
:10038000600FA500B010A00050129B00C013960093
:1003900040159100C0168C00C0188700901A82008A
:1003A000C01C7D00901E7800E0207300E0226E00EB
:1003B000F02469004027640040295F00802B5A0028
:1003C000D02D5500902F5000A0314B003033460007
:1003D000F034410060363C00C0373700F03832005E
:1003E000103A2D00003B2800F03B2300B03C1E00DB
:1003F000503D1900D03D1400203E0F00903E0A00F1
:10040000D03E0500F03F000070012C019001270153
:10041000B0012201C0011D01F001180110021301F9
:1004200030020E016002090190020401C002FF00C7
:100430000003FA004003F5008003F000D003EB0056
:100440002004E6007004E100E004DC004005D70071
:10045000C005D2004006CD00D006C8008007C3000A
:100460003008BE00F008B900C009B400B00AAF00FF
:10047000B00BAA00D00CA500000EA000500F9B00EE
:10048000C01096005012910000148C00C015870017
:10049000B0178200B0197D00D01B7800001E7300D9
:1004A00040206E0090226900F024640040275F0025
:1004B00090295A00E02B5500102E500020304B00A0
:1004C00010324600E033410090353C0010373700D1
:1004D00070383200A0392D00B03A2800A03B23002C
:1004E000603C1E00103D1900903D1400103E0F00AE
:1004F000703E0A00C03E0500003F000045313A2032
:100500000045303A20005A3A2000593A2000583A23
:1005100020004D53312C4D53322050696E730A0028
:10052000205A3A0020593A0020583A00656E647308
:10053000746F7073206869743A200024F4D43050CA
:10054000C38E20C2A24017828B7011127A910D8146
:100550006CD90AA861E108C7586607615143061EB5
:100560004B5D05C145A7041A411104093D9803716B
:100570003931034036DB0265339102D430540280B6
:100580002E1D02632CEE01752AC501B028A00110B2
:100590002781018F2564012B244B01E0223401AC1B
:1005A000211F018D200D01801FFC00841EED00978E
:1005B0001DDF00B81CD200E61BC600201BBC006477
:1005C0001AB200B219A8000A19A0006A189900D13D
:1005D00017910040178B00B516840031167E00B3CA
:1005E0001579003A157300C7146F0058146A00EEAD
:1005F0001366008813630025135E00C7125B006C4E
:1006000012570015125400C111510070114F0021F2
:10061000114B00D61049008D1047004610440002CF
:10062000104200C00F4000800F3E00420F3C000609
:100630000F3B00CB0E3800930E37005C0E350027C1
:100640000E3400F30D3200C10D3100900D3000600A
:100650000D2E00320D2D00050D2C00D90C2B00AEF7
:100660000C2900850C29005C0C2700350C27000E96
:100670000C2600E80B2400C40B2400A00B23007DF3
:100680000B23005A0B2100390B2100180B2000F816
:100690000A1F00D90A1E00BB0A1E009D0A1D008009
:1006A0000A1D00630A1C00470A1B002C0A1B0011CC
:1006B0000A1A00F7091A00DD091900C4091900AB6C
:1006C000091900920917007B091800630917004CEB
:1006D00009160036091600200916000A091500F54A
:1006E000081500E0081400CC081400B8081400A491
:1006F000081400900813007D0812006B08130058BE
:1007000008120046081200340811002308110012D4
:1007100008110001081100F0071000E0071000D0D8
:10072000071000C0071000B0070F00A107100091CC
:10073000070E0083070F0074070F0065070E0057B0
:10074000070E0049070E003B070D002E070E002084
:10075000070D0013070D0006070D00F9060C00ED4C
:10076000060D00E0060C00D4060C00C8060C00BC08
:10077000060C00B0060C00A4060B0099060C008DB8
:10078000060B0082060B0077060B006C060B00615F
:10079000060A0057060B004C060A0042060A0038FB
:1007A000060A002E060A0024060A001A060A00108D
:1007B00006090007060A00FD050900F4050900EB1B
:1007C000050900E2050900D9050900D0050900C79F
:1007D000050900BE050900B5050800AD050800A51E
:1007E0000509009C050800940508008C0508008494
:1007F0000508007C050800740508006C0507006505
:100800000508005D050700560508004E050700476E
:100810000507004005080038050700310507002AD4
:10082000050700230507001C050600160507000F35
:100830000507000805060002050700FB040600F591
:10084000040700EE040600E8040600E2040700DBEB
:10085000040600D5040600CF040600C9040600C340
:10086000040600BD040600B7040600B1040500AC90
:10087000040600A6040600A00405009B04060095DB
:10088000040500900406008A040500850405008024
:100890000406007A04050075040500700405006B69
:1008A00004050066040500610405005C04050057AA
:1008B000040500520405004D0405004804050043EA
:1008C0000405003E0404003A040500350405003028
:1008D0000404002C04050027040400230405001E62
:1008E0000404001A04040016040500110404000D99
:1008F000040400090405000404040000040400FCCE
:10090000030400F8030400F4030400F0030400EC03
:10091000030400E8030400E4030400E0030400DC33
:10092000030400D8030400D4030400D0030400CC63
:10093000030400C8030300C503030024F404D92002
:100940001BC40C5C0E9804C4095F0265077101F4B6
:1009500005F900FB04B30048048700C1036900588F
:1009600003550003034500BE023A008402310053E0
:10097000022A002902250004022000E4011C00C80C
:10098000011900AF011700980114008401130071D0
:100990000110006101100051010E0043010D0036ED
:1009A000010B002B010B0020010B00150109000CAD
:1009B00001090003010800FB000800F3000800EB38
:1009C000000700E4000600DE000600D8000600D2A2
:1009D000000600CC000500C7000500C2000500BDF0
:1009E000000400B9000400B5000400B1000400AD2B
:1009F000000400A9000400A5000300A20003009F5A
:100A00000004009B0003009800030095000200937F
:100A1000000300900003008D0002008B000300889B
:100A20000002008600020084000300810002007FB3
:100A30000002007D0002007B0002007900020077C6
:100A400000010076000200740002007200010071D3
:100A50000002006F0002006D0001006C0002006ADD
:100A600000010069000200670001006600010065E6
:100A700000010064000200620001006100010060EA
:100A80000001005F0002005D0001005C0001005BEE
:100A90000001005A000100590001005800010057F0
:100AA00000010056000100550001005400010053F0
:100AB00000000053000100520001005100010050ED
:100AC0000001004F0001004E0000004E0001004DEB
:100AD0000001004C0001004B0000004B0001004AE7
:100AE00000010049000100480000004800010047E3
:100AF00000010046000000460001004500000045DE
:100B000000010044000100430000004300010042D6
:100B100000000042000100410000004100010040CF
:100B20000001003F0000003F0001003E0000003EC9
:100B30000001003D0000003D0001003C0000003CC1
:100B40000000003C0001003B0000003B0001003AB7
:100B50000000003A000100390000003900010038AF
:100B600000000038000000380001003700000037A6
:100B7000000100360000003600000036000100359C
:100B80000000003500000035000100340000003492
:100B90000000003400010033000000330000003387
:100BA000000100320000003200000032000100317C
:100BB0000000003100000031000100300000003072
:100BC000000000300001002F0000002F0000002F67
:100BD0000000002F0001002E0000002E0000002E5B
:100BE0000001002D0000002D0000002D0000002D50
:100BF0000001002C0000002C0000002C0000002C44
:100C00000001002B0000002B0000002B0000002B37
:100C10000001002A0000002A0000002A0000002A2B
:100C2000000100290000002900000029000000291F
:100C30000000002900010028000000280000002812
:100C40000000002800000028000100270000002705
:100C500000000027000000270000002700010026F8
:100C600000000026000000260000002600000026EC
:100C700000010025000000250000002500000025DF
:100C800000000025000000250001002400000024D1
:100C900000000024000000240000002400010023C4
:100CA00000000023000000230000002300000023B8
:100CB00000000023000000230001002200000022A9
:100CC000000000220000002200000022000000229C
:100CD000000100210000002100000021000000218F
:100CE0000000002100000021000000210001002080
:100CF0000000002000000020000000200000002074
:100D00000000002000000020000000200001001F63
:100D10000000001F0000001F0000001F0000001F57
:100D20000000001F0000001F0001001E0000001E48
:100D30000000001E0000001E0000006563686F3A9E
:100D40000020746F6F206C6F6E6720657874727509
:100D500073696F6E2070726576656E7465640020CD
:100D6000636F6C6420657874727573696F6E207040
:100D7000726576656E746564006563686F3A0050ED
:100D800072696E7465722073746F7070656420642C
:100D9000756520746F206572726F72732E204669BC
:100DA0007820746865206572726F7220616E6420AD
:100DB000757365204D39393920746F2072657374ED
:100DC0006172742E202854656D706572617475723D
:100DD000652069732072657365742E2053657420D5
:100DE00069742061667465722072657374617274CF
:100DF000696E6729005072696E7465722068616C53
:100E00007465642E206B696C6C28292063616C6C9E
:100E1000656421006F6B00526573656E643A200053
:100E20002200556E6B6E6F776E20636F6D6D616E15
:100E3000643A2022007A5F6D61783A20007A5F6D13
:100E4000696E3A2000795F6D61783A2000795F6DB4
:100E5000696E3A2000785F6D61783A2000785F6DA6
:100E6000696E3A20005A3A00593A0020436F756E75
:100E70007420583A2000453A005A3A00593A00582E
:100E80003A004649524D574152455F4E414D453A11
:100E90004D61726C696E2056313B20537072696EE1
:100EA0007465722F6772626C206D61736875702053
:100EB000666F722067656E36204649524D57415223
:100EC000455F55524C3A687474703A2F2F77777794
:100ED0002E6D656E64656C2D70617274732E636F18
:100EE0006D2050524F544F434F4C5F56455253491B
:100EF0004F4E3A312E30204D414348494E455F54C4
:100F00005950453A4D656E64656C204558545255AC
:100F10004445525F434F554E543A310A0020423AFD
:100F20000020453A00543A0020573A0020453A0044
:100F3000543A002042403A0020403A00202F00203E
:100F4000423A00202F006F6B20543A002569206D33
:100F5000696E2C20256920736563005072696E7478
:100F600065722073746F7070656420647565207499
:100F70006F206572726F72732E20466978207468D4
:100F800065206572726F7220616E642075736520D2
:100F90004D39393920746F20726573746172742E03
:100FA000202854656D70657261747572652069736F
:100FB0002072657365742E205365742069742061F6
:100FC000667465722072657374617274696E6729E4
:100FD000006F6B004E6F204C696E65204E756D6220
:100FE0006572207769746820636865636B73756DDB
:100FF0002C204C617374204C696E653A20004E6F52
:1010000020436865636B73756D2077697468206C25
:10101000696E65206E756D6265722C204C6173740B
:10102000204C696E653A2000636865636B73756D6B
:10103000206D69736D617463682C204C617374203A
:101040004C696E653A20004C696E65204E756D6284
:101050006572206973206E6F74204C617374204C2C
:10106000696E65204E756D6265722B312C204C6166
:101070007374204C696E653A20004D313130002088
:1010800020506C616E6E657242756666657242795B
:101090007465733A20002046726565204D656D6F5A
:1010A00072793A2000417072203137203230313568
:1010B00000436F6D70696C65643A20004C756C7A02
:1010C000426F7400207C20417574686F723A200072
:1010D000323031332D30332D303600204C61737473
:1010E00020557064617465643A2000312E302E30D2
:1010F000004D61726C696E200020536F66747761D9
:10110000726520526573657400205761746368646A
:101110006F67205265736574002042726F776E208E
:101120006F7574205265736574002045787465721C
:101130006E616C20526573657400506F77657255EF
:101140007000737461727400FFFFFF0000A0400024
:1011500000A0400000803F000095430080894300CC
:10116000007A4300000000000000000000000000C2
:101170000095430080894300007A4300000000008E
:10118000000000000000006563686F3A004572725D
:101190006F723A000000090A02080B0C0D070603E3
:1011A000040100000000000000000000000000003A
:1011B000000000000000000000000000000000002F
:1011C00011100F00000000000000000000000000EF
:1011D00000000000000000000000010210202008B4
:1011E0000810204010204080020102010804020182
:1011F00001020408102040808040201008040201F1
:101200008004020180402010080402010804020149
:1012100001020408102040800102040810204080D0
:1012200005050505070508080808020202020A0A62
:101230000808040404040101010101010101030380
:10124000030303030303040707070C0C0C0C0C0C2B
:101250000C0C0202020206060606060606060B0B28
:101260000B0B0B0B0B0B00002000230026002900AA
:101270002C002F00320000010000030106010901CB
:1012800000002200250028002B002E003100340031
:1012900002010000050108010B01000021002400EB
:1012A00027002A002D003000330001010000040156
:1012B00007010A014E414E494E495459494E46CD07
:1012C000CCCC3D0AD7233C17B7D13877CC2B3295FD
:1012D00095E6241FB14F0A000020410000C84200DB
:1012E000401C4620BCBE4CCA1B0E5AAEC59D7400A5
:1012F00011241FBECFEFD1E2DEBFCDBF00E00CBF97
:1013000013E0A0E0B2E0E8E5F4EB00E00BBF02C0C0
:1013100007900D92A83DB107D9F71CE0A8EDB3E006
:1013200001C01D92A736B107E1F70E94624F0C94ED
:101330002A5A0C9400004F925F926F927F928F9284
:101340009F92AF92BF92CF92DF92EF92FF920F9354
:101350001F93CF93DF933C012CE034E081E090E0D9
:10136000F90105911491601671060CF055C09C01AD
:1013700021503109220F331F220F331FF901E65F7D
:10138000FB4FA590B490285F3B4FF901C591D491D4
:10139000FC01EE0FFF1FEE0FFF1FE65FFB4F859076
:1013A0009490B501882777FD8095982F0E94E95089
:1013B0006B017C01B3016C1B7D0B882777FD809549
:1013C000982F0E94E9502B013C01B4016A197B0956
:1013D000882777FD8095982F0E94E9509B01AC01EA
:1013E000C301B2010E941C534B015C01B8016C1B8C
:1013F0007D0B882777FD8095982F0E94E9509B01EF
:10140000AC01C501B4010E944E509B01AC01C70163
:10141000B6010E946E4F11C001962C5F3F4F8D3375
:10142000910509F09DCFEAEFF4E06591749188276A
:1014300077FD8095982F0E94E950DF91CF911F9101
:101440000F91FF90EF90DF90CF90BF90AF909F9063
:101450008F907F906F905F904F9008952F923F9262
:101460004F925F926F927F928F929F92AF92BF92B4
:10147000CF92DF92EF92FF920F931F93CF93DF9360
:10148000EC01662351F1E1E2F3E08491882341F01D
:101490009091C00095FFFCCF8093C6003196F5CFA8
:1014A00070E04AE050E083ED9BE00E94CD4AE7E126
:1014B000F2E08491882341F09091C00095FFFCCF29
:1014C0008093C6003196F5CF8091C00085FFFCCF98
:1014D0008AE08093C6000E94023A2CE233E081E069
:1014E00090E0F901A590B490CA15DB050CF055C049
:1014F0009C0121503109220F331F220F331FF901A4
:10150000E65DFC4F85909490285D3C4FF901059174
:101510001491FC01EE0FFF1FEE0FFF1FE65DFC4F65
:1015200025903490B401882777FD8095982F0E94EC
:10153000E9506B017C01BE01601B710B882777FDB0
:101540008095982F0E94E9502B013C01B101681948
:101550007909882777FD8095982F0E94E9509B0193
:10156000AC01C301B2010E941C532B013C01B50127
:10157000601B710B882777FD8095982F0E94E9509A
:101580009B01AC01C301B2010E944E509B01AC0112
:10159000C701B6010E946E4F11C001962C5F3F4FEC
:1015A0008833910509F09DCFE6E0F4E065917491F0
:1015B000882777FD8095982F0E94E950DF91CF9181
:1015C0001F910F91FF90EF90DF90CF90BF90AF9061
:1015D0009F908F907F906F905F904F903F902F9053
:1015E000089560E0809124049091250437DF609392
:1015F000200470932104809322049093230480910B
:101600001E0490911F0497DE60931A0470931B04CC
:1016100080931C0490931D048FB7F89410921904C2
:101620008FBF089520910D0230910E0240910F025C
:101630005091100260E070E08FE793E40E944E50FA
:101640006093F9037093FA038093FB039093FC0378
:10165000089597FF03C08091F20304C0FC01ED5090
:10166000FC4F808190E008952F923F924F925F92BD
:101670006F927F928F929F92AF92BF92CF92DF92A2
:10168000EF92FF920F931F93CF93DF9300D01F929F
:10169000CDB7DEB780911904882309F4A5C1A1DF75
:1016A000C0902004D0902104E0902204F090230404
:1016B0006091280470912904882777FD8095982FE0
:1016C0000E94E950A70196010E946D4F2B013C0139
:1016D00060930104709302048093030490930404C4
:1016E00020E030E040E251E40E944A5218160CF427
:1016F000E9C020E030E040E251ECC301B2010E94B9
:10170000475087FDDBC08091F8038111CCC0209148
:101710001102309112024091130250911402C30140
:10172000B2010E941C534B015C0160930D04709345
:101730000E0480930F0490931004209115043091AF
:1017400016044091170450911804C301B2010E947D
:101750006E4F2B013C010091FD031091FE03209080
:10176000FF03309000049801A1010E94475087FDBB
:1017700098C00091F9031091FA032090FB03309078
:10178000FC039801A101B201C3010E944A5218163C
:101790000CF487C08201C801D30180931504909393
:1017A0001604A0931704B093180420910D023091F1
:1017B0000E0240910F0250911002B801C3010E9425
:1017C0001C5369837A838B839C8360930904709391
:1017D0000A0480930B0490930C042091110430911F
:1017E00012044091130450911404C701B6010E94E1
:1017F0006D4F2091090230910A0240910B025091E5
:101800000C020E941C5320ED3CEC4CE45DE30E9472
:101810001C532B013C0123E333E343E75FE3609177
:1018200005047091060480910704909108040E94B9
:101830001C539B01AC01C301B2010E946E4F2B01EE
:101840003C01609305047093060480930704909311
:101850000804C0921104D0921204E0921304F09292
:10186000140429813A814B815C81C501B4010E9435
:101870006E4FA30192010E946D4F4B015C0120E06D
:1018800030E0A9010E94475087FD26C020E030E0EB
:1018900040E853E4C501B4010E944A521816FCF412
:1018A00014C0310178CF10921504109216041092D2
:1018B0001704109218041092F80329CF81E0809346
:1018C000F8030AC081E08093F803812C912CF0E8A2
:1018D000AF2EF3E4BF2E03C0812C912C54016091F4
:1018E000EE037091EF03882777FD8095982F0E9473
:1018F000E9509B01AC01C701B6010E944A5218167B
:101900001CF01092F3031AC0609101027091020260
:10191000882777FD8095982F0E94E9509B01AC01A4
:10192000C701B6010E94475087FFEBCFC501B40144
:101930000E94B650759567956093F3030E940F4D12
:101940000091F4031091F5032091F6033091F70311
:10195000601B710B820B930B6838734181059105F5
:1019600008F442C00E940F4D6093F4037093F50396
:101970008093F6039093F703C0901A04D0901B0451
:10198000E0901C04F0901D0420E030E040EA50E4B8
:10199000C701B6010E944A5218161CF520E030E03B
:1019A00046E153E4C701B6010E94475087FF19C0C2
:1019B0006091260470912704882777FD8095982FE1
:1019C0000E94E9509B01AC01C701B6010E944A5236
:1019D00087FD03C01092F20307C080E88093F203F2
:1019E00003C01092F20375980F900F900F900F9014
:1019F000DF91CF911F910F91FF90EF90DF90CF90EB
:101A0000BF90AF909F908F907F906F905F904F901E
:101A10003F902F9008950F931F93CF93DF931092D1
:101A2000FD031092FE031092FF0310920004209118
:101A30000D0230910E0240910F025091100260E0B1
:101A400070E08FE793E40E944E506093F903709327
:101A5000FA038093FB039093FC038091010180645F
:101A600080930101809101018061809301016D9A51
:101A70008091010180628093010187ED80937A005B
:101A800010927E0010927D0080917E008160809394
:101A90007E0080917E00826080937E0080917E0037
:101AA000846080937E0080E888BD80916E008460B1
:101AB00080936E006AEF70E080E090E00E943E4DFF
:101AC00085E090E09093EF038093EE0360E08091D7
:101AD000030290910402C2DC20E030E040EA50E4CE
:101AE0000E94475087FF0AC0809103029091040230
:101AF00040979093040280930302E8CF8AEF90E02E
:101B0000909302028093010260E08091F003909133
:101B1000F103A4DC20E030E04AE753E40E944A529B
:101B2000181654F48091F0039091F103409690932D
:101B3000F1038093F003E8CFC091EC03D091ED0363
:101B40008E01CE01F8DB609620E030E046E153E400
:101B50000E944A521816A4F30093EC031093ED036D
:101B6000DF91CF911F910F9108950895109229044C
:101B70001092280410922704109226041092F30366
:101B80009FB7F894E2E0F1E080818F7B80839FBF74
:101B900010922B0410922A041092F4039FB7F89429
:101BA000E2E0F1E080818F7E80839FBF1092270466
:101BB000109226041092F203759808952F923F9286
:101BC0004F925F926F927F928F929F92AF92BF924D
:101BD000CF92DF92EF92FF920F931F93CF93DF93F9
:101BE000CDB7DEB7E3970FB6F894DEBF0FBECDBF1B
:101BF0006C8F7D8F8E8F9F8F5BAB4AAB3CA72BA7E3
:101C00000E940F4D69A37AA38BA39CA32AA93BA989
:101C1000223031051CF4EEE8F2E017C0E1EAF2E010
:101C20008191882339F09091C00095FFFCCF80937B
:101C3000C600F6CF8091C00085FFFCCF2BC29091EB
:101C4000C00095FFFCCF8093C60081918111F7CF32
:101C50008091C00085FFFCCF8AE08093C60086DFBC
:101C60004AA95BA980E857FF03C08093F20305C02F
:101C7000EAA9FBA9ED50FC4F808389A19AA1ABA1F1
:101C8000BCA1898B9A8BAB8BBC8B8D879E87AF87D2
:101C9000B88B1D8290E4998FACE1AA8FB6E4BB8F1C
:101CA0001D8A1E8A1F8A188E20E830E040E050E02E
:101CB00029833A834B835C8370E8472E512C612C37
:101CC000712C1DA21EA21FA218A631E038A31C86EB
:101CD0001B86312C00E010E0212C4AA95BA94D5055
:101CE0005C4F5AA749A7E9E1F3E054915DA7E4E10D
:101CF000F3E084918EA7EDE0F3E094919FA7E6E0F6
:101D0000F3E0A491A8ABE0E0F3E0B491B9ABEAA9A9
:101D1000FBA9EE0FFF1FEE0FFF1FE05EFB4FFA87E0
:101D2000E98780911904882309F4E1C05ADC2AA9C3
:101D30003BA937FF09C030901A0400911B04109191
:101D40001C0420901D040BC0A985BA853C901196F7
:101D50000C91119712961C91129713962C90232D8B
:101D6000302F412F522D6D897E898F89988D0E9449
:101D70004A52181624F03D8A0E8B1F8B288E232D75
:101D8000302F412F522D6D81798D8A8D9B8D0E9430
:101D9000475087FD04C03D82098F1A8F2B8EB8A152
:101DA000BB2309F451C02C8D3D8D4E8D5F8D632D6D
:101DB000702F812F922D0E944A5218160CF097C056
:101DC0000E940F4D29893A894B895C89621B730BEC
:101DD000840B950B693873418105910508F487C020
:101DE000D301C20129813A814B815C81821B930B13
:101DF000A40BB50B4AA95BA9B595A79597958795AF
:101E000057FF03C08093F20303C0E9A5FAA58083BE
:101E10000E940F4D6D877E878F87988B9B01AC0149
:101E200089899A89AB89BC89281B390B4A0B5B0BC2
:101E30002DA33EA34FA358A79C8D9D8BAD8DAE8B3C
:101E4000BE8DBF8BEF8DE88F2C8D3D8D4E8D5F8DC0
:101E5000632D702F812F922D0E94475087FFF5C26E
:101E60000E940F4D2D853E854F855889621B730B4F
:101E7000840B950B693873418105910508F4E5C21F
:101E80000E940F4D698B7A8B8B8B9C8BDC01CB0175
:101E90002D853E854F855889821B930BA40BB50B6E
:101EA0004B855C85452B09F011C189819A81AB81F5
:101EB000BC81840D951DA61DB71DEAA9FBA9B5958A
:101EC000A79597958795F7FFBCC28093F2032B8562
:101ED0003C852F5F3F4F3C872B873C8D3D834D8D4D
:101EE000498F5E8D5A8F8F8D8B8F91E098A320E064
:101EF00030E040EA51E46C8D7D8D8E8D9F8D0E9487
:101F00006E4F9B01AC01632D702F812F922D0E948B
:101F10004A52181694F4E2EBF2E08491882341F0DF
:101F20009091C00095FFFCCF8093C6003196F5CF0D
:101F30008091C00085FFFCCFADC00E940F4D29A14C
:101F40003AA14BA15CA1621B730B840B950B613D05
:101F500077408105910508F450C04AA95BA957FF55
:101F600010C0E090F203F12CECEAF2E084918823B7
:101F7000C9F09091C00095FFFCCF8093C6003196C8
:101F8000F5CFA9A5BAA5EC90F12CE6EAF2E0849190
:101F9000882341F09091C00095FFFCCF8093C6004C
:101FA0003196F5CF22E030E0432D502F612F722D76
:101FB00083ED9BE00E94994BE2EAF2E08491882352
:101FC00041F09091C00095FFFCCF8093C600319600
:101FD000F5CF4AE050E0B70183ED9BE00E94CD4A87
:101FE0008091C00085FFFCCF8AE08093C6000E94EC
:101FF0000F4D69A37AA38BA39CA30E940F4D6B0185
:102000007C010E940F4D89889A88AB88BC882D85F9
:102010003E854F855889820E931EA41EB51EC81892
:10202000D908EA08FB08C60ED71EE81EF91E31E8DB
:10203000C3163FE4D30632E1E306F10490F0E5E88D
:10204000F2E08491882341F09091C00095FFFCCF8D
:102050008093C6003196F5CF8091C00085FFFCCFFC
:1020600019C04B855C858BA59CA5841795070CF042
:1020700058CEE4E3F2E08491882341F09091C000CF
:1020800095FFFCCF8093C6003196F5CF8091C000BC
:1020900085FFFCCF8AE08093C600E3960FB6F894E4
:1020A000DEBF0FBECDBFDF91CF911F910F91FF908B
:1020B000EF90DF90CF90BF90AF909F908F907F90E8
:1020C0006F905F904F903F902F9008958DA09EA0AD
:1020D000AFA0B8A4880E991EAA1EBB1E2DA13EA1BA
:1020E0004FA158A5281B390B4A0B5B0BCA01B9013C
:1020F00029813A814B815C810E94E853A5019401BA
:102100000E942C54240D351D461D571D24313105C8
:102110004105510504F129013A013DEE43165104F0
:10212000610471042CF04CEE442E512C612C712C66
:1021300041E84416510461047104DCF08FEF90E033
:10214000A0E0B0E084199509A609B70989839A83AC
:10215000AB83BC8312C034E1432E512C612C712C13
:1021600024E130E040E050E029833A834B835C83F4
:1021700004C049825A826B827C828DA5E9E1F3E03A
:10218000882349F09091C00095FFFCCF8093C60052
:1021900031968491F5CF2AE030E0B301A20183EDBE
:1021A0009BE00E94AA4A8EA5E4E1F3E0882349F06F
:1021B0009091C00095FFFCCF8093C600319684912A
:1021C000F5CF2AE030E049815A816B817C8183ED33
:1021D0009BE00E94AA4A8FA5EDE0F3E0882349F036
:1021E0009091C00095FFFCCF8093C60031968491FA
:1021F000F5CF22E030E04D81598D6A8D7B8D83EDE6
:102200009BE00E94994B88A9E6E0F3E0882349F01F
:102210009091C00095FFFCCF8093C60031968491C9
:10222000F5CF22E030E04D895E896F89788D83EDAE
:102230009BE00E94994B8091C00085FFFCCF8AE013
:102240008093C6004B855C85433051050CF42DCE40
:1022500069817A818B819C810E94E95020E030E085
:1022600040E850E40E941C536B017C012D81398DA4
:102270004A8D5B8D6D897E898F89988D0E946D4F07
:1022800020ED3FE049E450E40E941C5320E030E0A0
:1022900040E05FE30E941C539B01AC01C701B60103
:1022A0000E944E506B017C01C501B4010E94E950AF
:1022B00020E030E04AE754E40E944E504B015C01BC
:1022C00089A9E0E0F3E0882349F09091C00095FFF0
:1022D000FCCF8093C60031968491F5CF22E030E0A8
:1022E000B701A60183ED9BE00E94994BEAEFF2E073
:1022F0008491882341F09091C00095FFFCCF80939A
:10230000C6003196F5CF22E030E0B501A40183ED9F
:102310009BE00E94994B8091C00085FFFCCF8AE032
:102320008093C6002AE939E949E15FE3C701B601B4
:102330000E941C536B017C019B01AC010E946E4FFB
:10234000A50194010E944E506D837E838F839887F0
:10235000A5019401C701B6010E941C5320E030E0A2
:1023600040E05EE30E941C534B015C01EDEEF2E0A5
:102370008491882341F09091C00095FFFCCF809319
:10238000C6003196F5CF8091C00085FFFCCF8AE072
:102390008093C600E7EEF2E08491882341F09091AB
:1023A000C00095FFFCCF8093C6003196F5CF22E0A8
:1023B00030E0B701A60183ED9BE00E94994B80912C
:1023C000C00085FFFCCF8AE08093C600E1EEF2E01A
:1023D0008491882341F09091C00095FFFCCF8093B9
:1023E000C6003196F5CF22E030E04D815E816F81ED
:1023F000788583ED9BE00E94994B8091C00085FF1A
:10240000FCCF8AE08093C600EBEDF2E08491882354
:1024100041F09091C00095FFFCCF8093C6003196AB
:10242000F5CF22E030E0B501A40183ED9BE00E94EE
:10243000994B8091C00085FFFCCF8AE08093C60055
:1024400034CDE9A5FAA5808342CD18A250CDCF9313
:10245000C82F8CDB0E94CA3A811130C0E1E2F3E060
:102460009491992341F08091C00085FFFCCF909317
:10247000C6003196F5CF6C2F70E04AE050E083ED56
:102480009BE00E94CD4A8091C00085FFFCCF8AE08E
:102490008093C600EAEEF1E08491882341F09091A8
:1024A000C00095FFFCCF8093C6003196F5CF809198
:1024B000C00085FFFCCF8AE08093C600CF910C94CA
:1024C0008F3ACF93C82F52DB0E94CA3A811130C095
:1024D000E1E2F3E09491992341F08091C00085FFFF
:1024E000FCCF9093C6003196F5CF6C2F70E04AE098
:1024F00050E083ED9BE00E94CD4A8091C00085FFB3
:10250000FCCF8AE08093C600EDEBF1E08491882354
:1025100041F09091C00095FFFCCF8093C6003196AA
:10252000F5CF8091C00085FFFCCF8AE08093C60084
:10253000CF910C948F3A75980E94CA3A811121C0AC
:10254000E1E2F3E08491882341F09091C00095FF8F
:10255000FCCF8093C6003196F5CFE3E8F1E084919B
:10256000882341F09091C00095FFFCCF8093C60076
:102570003196F5CF8091C00085FFFCCF8AE0809333
:10258000C6000C948F3A1F920F920FB60F9211242F
:102590000BB60F922F933F934F935F936F937F935D
:1025A0008F939F93AF93BF93EF93FF93809100021C
:1025B000811114C08091F3038093EB03882341F0D1
:1025C0009FB7F894809102018064809302019FBFBD
:1025D0008091F2038093EA038111759A9091EB0345
:1025E00080910002891740F09FB7F8948091020112
:1025F0008F7B809302019FBF9091EA03809100023C
:10260000891708F07598809100028F5F8F7780930B
:1026100000028091E90390E08830910508F082C0C3
:10262000FC01EE58FF4F0C94485410927B0080E45C
:1026300080937C0080917A00806480937A0081E0AE
:1026400019C020917800309179008091E503909134
:10265000E603A091E703B091E803820F931FA11D49
:10266000B11D8093E5039093E603A093E703B09335
:10267000E80382E08093E90355C010927B0082E476
:1026800080937C0080917A00806480937A0083E05C
:10269000F1CF20917800309179008091E103909101
:1026A000E203A091E303B091E403820F931FA11D05
:1026B000B11D8093E1039093E203A093E303B093F1
:1026C000E40384E0D7CF10927B0081E480937C0008
:1026D00080917A00806480937A0085E0CBCF20914E
:1026E0007800309179008091DD039091DE03A09114
:1026F000DF03B091E003820F931FA11DB11D8093F2
:10270000DD039093DE03A093DF03B093E00386E044
:10271000B1CF87E0AFCF1092E9038091DC038F5FE8
:102720008093DC038091DC03803108F463C08091E6
:102730001904811110C08091E5039091E6039093F4
:102740002504809324048091E1039091E203909307
:102750001F0480931E0481E0809319041092DC030F
:102760001092E5031092E6031092E7031092E8033B
:102770001092DD031092DE031092DF031092E0034B
:102780001092D8031092D9031092DA031092DB034F
:102790001092E1031092E2031092E3031092E4031B
:1027A00020912404309125048091F0039091F1034D
:1027B0008217930714F080E04ADE209124043091C0
:1027C000250480910302909104022817390714F020
:1027D00080E077DE20911E0430911F048091EC038D
:1027E0009091ED03821793072CF01092270410921A
:1027F0002604A1DEFF91EF91BF91AF919F918F9140
:102800007F916F915F914F913F912F910F900BBEF0
:102810000F900FBE0F901F90189580914204811168
:1028200009C080914104811105C08091400481114B
:1028300001C00895EBE3FDE08491882341F090917D
:10284000C00095FFFCCF8093C6003196F5CFECE237
:10285000F5E08491882341F09091C00095FFFCCF72
:102860008093C6003196F5CF809142048823D1F041
:102870006091430470914404809145049091460412
:102880000E94E9502091AB093091AC094091AD090B
:102890005091AE090E944E50AB01BC0188E295E018
:1028A0000E949132809141048823D1F060914704C5
:1028B000709148048091490490914A040E94E95023
:1028C0002091AF093091B0094091B1095091B209FE
:1028D0000E944E50AB01BC0184E295E00E9491320F
:1028E000809140048823D1F060914B0470914C0496
:1028F00080914D0490914E040E94E9502091B309BB
:102900003091B4094091B5095091B6090E944E50DA
:10291000AB01BC0180E295E00E9491328091C00041
:1029200085FFFCCF8AE08093C6001092420410928B
:102930004104109240040895109242041092410400
:10294000109240040895809319020895EFE6F0E094
:1029500080818260808308951F920F920FB60F923C
:1029600011240BB60F920F931F932F933F934F9306
:102970005F936F937F938F939F93AF93BF93EF93E7
:10298000FF938091710490917204892B09F07DC1AD
:102990009091790480917804981771F0E09178040F
:1029A0008DE4E89FF0011124E658FB4FDF01A45BA2
:1029B000BF4F81E08C9302C0E0E0F0E0F09372043E
:1029C000E0937104309709F45AC1DF01A45BBF4F53
:1029D00081E08C9310925404109255041092560486
:1029E0001092570460AD71AD61349CE9790728F409
:1029F00061329EE4790748F002C060E47CE9769594
:102A000067957695679584E007C0613197E279070D
:102A100030F07695679582E08093510407C08093EB
:102A200051046032710510F460E270E06052710987
:102A3000611588E07807D0F0872F9927880F991FB4
:102A4000880F991F855C964FFC01329645915491F1
:102A5000AA27659F9001649F210D3A1F06942A1FA3
:102A60003A1F1124FC01859194911DC09B0136955C
:102A700027952C7F255C3A4FF901859194912E5F23
:102A80003F4FF90145915491FB01E770FF274E9F9D
:102A900090014F9F300D5E9F300D112413E036954D
:102AA00027951A95E1F7821B930B84369105A0F4C4
:102AB000EBECF2E08191882339F09091C00095FF12
:102AC000FCCF8093C600F6CF4AE050E083ED9BE058
:102AD0000E940A4B84E690E09093500480934F0448
:102AE000E0917104F091720464AD75AD709353047C
:102AF0006093520461349CE9790728F461328EE4D2
:102B0000780748F002C060E47CE976956795769591
:102B1000679584E007C0613197E2790730F07695D8
:102B2000679582E08093510408C081E0809351044E
:102B30006032710510F460E270E060527109611555
:102B400088E07807E0F0872F9927880F991F880F72
:102B5000991F855C964FFC01329625913491AA27E6
:102B6000639FA001629F410D5A1F06944A1F5A1F7E
:102B70001124FC0125913491241B350B1EC0CB017F
:102B8000969587958C7F855C9A4FFC0125913491B1
:102B90000296FC0145915491FB01E770FF274E9F7F
:102BA000C0014F9F900D5E9F900D112443E09695BC
:102BB00087954A95E1F7281B390B24363105A0F497
:102BC000EBECF2E08191882339F09091C00095FF01
:102BD000FCCF8093C600F6CF4AE050E083ED9BE047
:102BE0000E940A4B24E630E0C901A0E0B0E08093E7
:102BF000580490935904A0935A04B0935B04309303
:102C0000890020938800E0917104F091720480891A
:102C10009189A289B389B695A79597958795B0951F
:102C2000A095909581959F4FAF4FBF4F80936C04B7
:102C300090936D04A0936E04B0936F048093680426
:102C400090936904A0936A04B0936B048093640426
:102C500090936504A0936604B09367048093600426
:102C600090936104A0936204B093630410925C0497
:102C700010925D0410925E0410925F0406C080ED15
:102C800097E09093890080938800E0917104F0911F
:102C90007204309709F488C580A1809370049FB7AF
:102CA00080FF48C0F89480910B018D7F80930B01C9
:102CB0009FBF8FEF8093150280911902882309F43A
:102CC0007EC023B131E026FB222720F9232779F1AA
:102CD00080913F04882359F1E0917104F0917204CE
:102CE00080819181A281B381181619061A061B06EC
:102CF000F4F480912A0490912B04A0912C04B091BB
:102D00002D048093430490934404A0934504B0930E
:102D100046043093420480899189A289B3898093C3
:102D20005C0490935D04A0935E04B0935F042093D1
:102D30003F0445C0F89480910B01826080930B01A1
:102D40009FBF31E030931502809119028823B9F1B9
:102D500020B122FB222720F9232779F180913E041C
:102D6000882359F1E0917104F0917204808191817E
:102D7000A281B381181619061A061B06F4F4809175
:102D80002A0490912B04A0912C04B0912D048093DF
:102D9000430490934404A0934504B09346043093B5
:102DA000420480899189A289B38980935C049093BD
:102DB0005D04A0935E04B0935F0420933E04809171
:102DC00070049FB781FF48C0F89480910B01816027
:102DD00080930B019FBF8FEF8093160280911902A1
:102DE000882309F47DC023B131E025FB222720F997
:102DF000232779F180913D04882359F1E0917104F2
:102E0000F091720484819581A681B7811816190604
:102E10001A061B06F4F480912E0490912F04A091C1
:102E20003004B09131048093470490934804A093F8
:102E30004904B0934A043093410480899189A2895E
:102E4000B38980935C0490935D04A0935E04B09377
:102E50005F0420933D0444C0F89480910B018E7F61
:102E600080930B019FBF31E03093160280911902CD
:102E70008823B1F120B126952170232779F1809123
:102E80003C04882359F1E0917104F091720484812B
:102E90009581A681B781181619061A061B06F4F447
:102EA00080912E0490912F04A0913004B0913104B0
:102EB0008093470490934804A0934904B0934A0434
:102EC0003093410480899189A289B38980935C04FD
:102ED00090935D04A0935E04B0935F0420933C0440
:102EE000809170049FB782FF47C0F89480910B01D6
:102EF0008B7F80930B019FBF8FEF80931702809190
:102F00001902882309F47DC023B131E02295217094
:102F1000232779F180913B04882359F1E0917104D2
:102F2000F091720480859185A285B38518161906E3
:102F30001A061B06F4F48091320490913304A09198
:102F40003404B091350480934B0490934C04A093C7
:102F50004D04B0934E043093400480899189A28936
:102F6000B38980935C0490935D04A0935E04B09356
:102F70005F0420933B0445C0F89480910B0184606A
:102F800080930B019FBF31E03093170280911902AB
:102F90008823B9F126B12095221F2227221F79F11B
:102FA00080913A04882359F1E0917104F091720400
:102FB00080859185A285B385181619061A061B0609
:102FC000F4F48091320490913304A0913404B091D0
:102FD000350480934B0490934C04A0934D04B0931C
:102FE0004E043093400480899189A289B3898093EB
:102FF0005C0490935D04A0935E04B0935F042093FF
:103000003A04809170049FB783FF09C0F8948091BF
:103010000B01806480930B019FBF8FEF08C0F89471
:1030200080910B018F7B80930B019FBF81E0809388
:10303000180220E08091510428170CF0ADC1809156
:10304000C00087FF19C03091C6004091540C5091C8
:10305000550CCA0101968F7799276091560C709193
:10306000570C8617970741F0FA01EC52F44F308362
:103070009093550C8093540CE0917104F09172047C
:1030800080916C0490916D04A0916E04B0916F04D6
:103090004081518162817381840F951FA61FB71FE4
:1030A00080936C0490936D04A0936E04B0936F04AE
:1030B000181619061A061B06CCF5409AE091710401
:1030C000F091720480916C0490916D04A0916E0453
:1030D000B0916F044089518962897389841B950B73
:1030E000A60BB70B80936C0490936D04A0936E04B1
:1030F000B0936F044091150280912A0490912B04A3
:10310000A0912C04B0912D04552747FD5095652FB3
:10311000752F840F951FA61FB71F80932A049093C5
:103120002B04A0932C04B0932D044098E0917104DB
:10313000F09172048091680490916904A0916A04EE
:10314000B0916B044481558166817781840F951F0E
:10315000A61FB71F8093680490936904A0936A0424
:10316000B0936B04181619061A061B06CCF5419A83
:10317000E0917104F0917204809168049091690467
:10318000A0916A04B0916B04408951896289738966
:10319000841B950BA60BB70B80936804909369046E
:1031A000A0936A04B0936B044091160280912E04A0
:1031B00090912F04A0913004B0913104552747FD20
:1031C0005095652F752F840F951FA61FB71F8093ED
:1031D0002E0490932F04A0933004B09331044198AF
:1031E000E0917104F09172048091640490916504FF
:1031F000A0916604B091670440855185628573850E
:10320000840F951FA61FB71F8093640490936504D5
:10321000A0936604B0936704181619061A061B06D5
:10322000CCF5429AE0917104F091720480916404AB
:1032300090916504A0916604B0916704408951891A
:1032400062897389841B950BA60BB70B809364046A
:1032500090936504A0936604B093670440911702AD
:103260008091320490913304A0913404B0913504DC
:10327000552747FD5095652F752F840F951FA61F65
:10328000B71F8093320490933304A0933404B09317
:1032900035044298E0917104F091720480916004C9
:1032A00090916104A0916204B091630444855585B6
:1032B00066857785840F951FA61FB71F80936004CE
:1032C00090936104A0936204B093630418161906E6
:1032D0001A061B06CCF5439AE0917104F091720432
:1032E0008091600490916104A0916204B0916304A4
:1032F0004089518962897389841B950BA60BB70B92
:103300008093600490936104A0936204B09363047B
:10331000409118028091360490913704A0913804AE
:10332000B0913904552747FD5095652F752F840FAF
:10333000951FA61FB71F8093360490933704A09360
:103340003804B0933904439880915C0490915D04F3
:10335000A0915E04B0915F040196A11DB11D809300
:103360005C0490935D04A0935E04B0935F0440916D
:103370005C0450915D0460915E0470915F04E09183
:103380007104F091720480899189A289B3894817E8
:1033900059076A077B07B0F040915C0450915D04C7
:1033A00060915E0470915F04E0917104F091720489
:1033B00084899589A689B78984179507A607B707D1
:1033C00018F4DAC02F5F36CE40915804509159045A
:1033D00060915A0470915B04048D158D268D378D94
:1033E000AA27419FB12D529FC001629F900D619FFE
:1033F000800D911D429FB00D811D9A1F519FB00DF0
:10340000811D9A1F609FB00D811D9A1F509FB10DA5
:103410008A1F9A1FB6958A1F9A1F112444AD55AD75
:10342000480F591F509353044093520480AD91ADFF
:10343000A2ADB3AD60E070E084179507A607B707AB
:1034400020F490935304809352046091520470913D
:10345000530461349CE9790728F461328EE47807DB
:1034600048F002C060E47CE97695679576956795AB
:1034700084E007C0613197E2790730F0769567956F
:1034800082E08093510408C081E08093510460324F
:10349000710510F460E270E060527109611588E016
:1034A0007807E0F0872F9927880F991F880F991FB9
:1034B000855C964FFC01329625913491AA27639F33
:1034C000A001629F410D5A1F06944A1F5A1F1124E2
:1034D000FC0125913491241B350B1EC0CB01969520
:1034E00087958C7F855C9A4FFC01259134910296DB
:1034F000FC0145915491FB01E770FF274E9FC001ED
:103500004F9F900D5E9F900D1124F3E09695879547
:10351000FA95E1F7281B390B24363105A0F4EBECC2
:10352000F2E08191882339F09091C00095FFFCCFA3
:103530008093C600F6CF4AE050E083ED9BE00E9406
:103540000A4B24E630E03093890020938800809174
:10355000580490915904A0915A04B0915B04820FD1
:10356000931FA11DB11D8093580490935904A093FB
:103570005A04B0935B04F3C040915C0450915D0425
:1035800060915E0470915F04808D918DA28DB38DEA
:1035900084179507A607B70708F0D9C040915404CF
:1035A000509155046091560470915704048D158D07
:1035B000268D378DAA27419FB12D529FC001629F52
:1035C000900D619F800D911D429FB00D811D9A1F2E
:1035D000519FB00D811D9A1F609FB00D811D9A1FD4
:1035E000509FB10D8A1F9A1FB6958A1F9A1F1124EA
:1035F0002091520430915304E05CFF4F28173907A3
:1036000018F42081318102C0281B390B80819181FF
:10361000A281B381A90160E070E0481759076A07E9
:103620007B0708F49C0121349CE9390728F42132F6
:103630008EE4380748F002C020E43CE9369527952F
:103640003695279584E007C0213197E2390730F09D
:103650003695279582E08093510408C081E08093DD
:1036600051042032310510F420E230E0B9016052FB
:103670007109611588E07807E0F0872F9927880F96
:10368000991F880F991F855C964FFC0132964591D2
:103690005491AA27659F9001649F210D3A1F0694BB
:1036A0002A1F3A1F1124FC0145915491421B530BD0
:1036B0001EC0CB01969587958C7F855C9A4FFC0147
:1036C000459154910296FC0125913491FB01E770DC
:1036D000FF272E9FC0012F9F900D3E9F900D11241C
:1036E00033E0969587953A95E1F7481B590B443698
:1036F0005105A0F4EBECF2E08191882339F0909130
:10370000C00095FFFCCF8093C600F6CF4AE050E0A2
:1037100083ED9BE00E940A4B44E650E05093890001
:10372000409388008091540490915504A0915604D0
:10373000B0915704840F951FA11DB11D80935404AF
:1037400090935504A0935604B093570408C08091F9
:103750004F04909150049093890080938800409189
:103760005C0450915D0460915E0470915F04E0918F
:103770007104F091720480899189A289B3894817F4
:1037800059076A077B0780F0109272041092710447
:103790009091790480917804981731F080917804A1
:1037A0008F5F8F7080937804FF91EF91BF91AF91FD
:1037B0009F918F917F916F915F914F913F912F9149
:1037C0001F910F910F900BBE0F900FBE0F901F9087
:1037D00018959091790480917804981729F00E94A7
:1037E000340B0E942F3AF5CF0895CF93DF93EFB7B4
:1037F000F894EC0188819981AA81BB8180932A0485
:1038000090932B04A0932C04B0932D04EB0188819A
:103810009981AA81BB8180932E0490932F04A09359
:103820003004B0933104EA0188819981AA81BB8177
:103830008093320490933304A0933404B0933504FE
:10384000E90188819981AA81BB8180933604909394
:103850003704A0933804B0933904EFBFDF91CF91C0
:1038600008952FB7F894FC0180819181A281B381E2
:103870008093360490933704A0933804B0933904AE
:103880002FBF08952FB7F89494E0899FF001112479
:10389000E65DFB4F60817181828193812FBF089526
:1038A00098DF179A169A159A149A0895CF93DF9372
:1038B000D82FC62F60E086E20E944C4EDEBD0DB4CC
:1038C00007FEFDCF8EB5CEBD0DB407FEFDCF8EB584
:1038D00061E086E2DF91CF910C944C4ECF93DF9361
:1038E00000D01F921F92CDB7DEB795E0EFE4F2E073
:1038F000DE01119601900D929A95E1F7E1E0F0E07A
:10390000EC0FFD1FE80FF11D808190E00F900F90EC
:103910000F900F900F90DF91CF91C8CFFF920F9330
:103920001F93CF93DF9300D01F921F92CDB7DEB7C6
:1039300085E0E4E5F2E0DE01119601900D928A95B2
:10394000E1F70E94B34C61E086E20E94134E8E01C3
:103950000F5F1F4FF12CF80161918F0170E08F2DE7
:10396000BDDFF394F5E0FF12F6CF0F900F900F90AC
:103970000F900F90DF91CF911F910F91FF900895BD
:10398000CF93C42F67FD2BC08230B9F028F4882371
:1039900041F0813061F023C08330A9F08430C9F058
:1039A0001EC088E20E944C4EC7FF28C038C085E484
:1039B0000E944C4EC7FF25C032C084E40E944C4E8A
:1039C000C7FF22C02CC081E40E944C4EC7FF1FC01D
:1039D00026C08FE30E944C4EC7FF1CC020C0C7FD0D
:1039E0001EC0823089F028F4882341F0813049F0EC
:1039F00016C0833061F0843069F011C06C2F89E209
:103A00000BC06C2F87E208C06C2F83E405C06C2FBD
:103A100082E402C06C2F80E4CF910C944C4ECF9185
:103A20000895643079F028F4613041F0623041F05B
:103A30000895683051F0603141F0089540E003C0CE
:103A400040E004C041E060E002C041E061E098CFA6
:103A5000FF920F931F93CF93DF9300D01F921F927B
:103A6000CDB7DEB785E0E9E5F2E0DE011196019021
:103A70000D928A95E1F761E089E20E94134E61E0C0
:103A800087E20E94134E61E083E40E94134E61E0DE
:103A900082E40E94134E61E080E40E94134E8E0186
:103AA0000F5F1F4FF12CF80161918F018F2DB9DF4E
:103AB000F394F5E0FF12F7CF0F900F900F900F9057
:103AC0000F90DF91CF911F910F91FF90089526DF06
:103AD000BFDFEAE0F1E080818260808380818160E5
:103AE0008083808184608083808180648083808102
:103AF000806880830F9A179A0E9A169A0D9A159AD3
:103B00000C9A149A0B9A139A26982E9A25982D9A05
:103B100024982C9A0A98129A0998119A3F98479AD1
:103B2000389A4098179A399A4198169A3A9A429830
:103B3000159A3B9A4398149A3C9A4498A1E8B0E0AD
:103B40008C918F7E8C938C9188608C93E0E8F0E070
:103B500080818D7F808380818E7F808380818F7341
:103B6000808380818F7C80838C91887F82608C931E
:103B700080E090E490938900809388001092850003
:103B800010928400EFE6F0E080818260808381E023
:103B90008093190278940895E2E1F5E084918823F6
:103BA00041F09091C00095FFFCCF8093C600319604
:103BB000F5CFEEE0F5E08491882341F09091C000CC
:103BC00095FFFCCF8093C6003196F5CF88E20E9426
:103BD000814E4AE050E0BC0183ED9BE00E94CD4A5B
:103BE00089E20E94814E4AE050E0BC0183ED9BE0F7
:103BF0000E94CD4A8091C00085FFFCCF8AE080936F
:103C0000C600EAE0F5E08491882341F09091C0007D
:103C100095FFFCCF8093C6003196F5CF85E40E94D6
:103C2000814E4AE050E0BC0183ED9BE00E94CD4A0A
:103C300087E20E94814E4AE050E0BC0183ED9BE0A8
:103C40000E94CD4A8091C00085FFFCCF8AE080931E
:103C5000C600E6E0F5E08491882341F09091C00031
:103C600095FFFCCF8093C6003196F5CF84E40E9487
:103C7000814E4AE050E0BC0183ED9BE00E94CD4ABA
:103C800083E40E94814E4AE050E0BC0183ED9BE05A
:103C90000E94CD4A8091C00085FFFCCF8AE08093CE
:103CA000C600E1E0F5E08491882341F09091C000E6
:103CB00095FFFCCF8093C6003196F5CF81E40E943A
:103CC000814E4AE050E0BC0183ED9BE00E94CD4A6A
:103CD00082E40E94814E4AE050E0BC0183ED9BE00B
:103CE0000E94CD4A8091C00085FFFCCF8AE080937E
:103CF000C600ECEFF4E08491882341F09091C0007D
:103D000095FFFCCF8093C6003196F5CF8FE30E94DC
:103D1000814E4AE050E0BC0183ED9BE00E94CD4A19
:103D200080E40E94814E4AE050E0BC0183ED9BE0BC
:103D30000E94CD4A8091C00085FFFCCF8AE080932D
:103D4000C60008952F923F924F925F926F927F929A
:103D50008F929F92AF92BF92CF92DF92EF92FF929B
:103D60000F931F93CF93DF93CDB7DEB768970FB64E
:103D7000F894DEBF0FBECDBF1C012A013B014801F4
:103D80005901DC01D8966D917D918D919C91DB97C5
:103D90000E94E7506B017C01A30192010E941C5319
:103DA0000E9434500E94BB506D877E878F87988B0E
:103DB000A5019401C701B6010E941C530E94345012
:103DC0000E94BB50698B7A8B8B8B9C8B2D853E859B
:103DD0004F855889283731054105510540F488E75A
:103DE00090E0A0E0B0E08D879E87AF87B88B2989EF
:103DF0003A894B895C89283731054105510540F4E2
:103E000088E790E0A0E0B0E0898B9A8BAB8BBC8B0D
:103E100091012C5B3F4FD9018D919D910D90BC91EB
:103E2000A02D8D839E83AF83B887BC01CD010E94F6
:103E3000E95069837A838B839C83F10164AD75AD0E
:103E400086AD97AD0E94E75069877A878B879C87FC
:103E500020E030E0A90169817A818B819C810E94F8
:103E60004750882339F1A7019601C701B6010E9486
:103E70001C534B015C0129853A854B855C85CA0141
:103E8000B9010E941C539B01AC01C501B4010E9401
:103E90006D4F4B015C0129813A814B815C81CA01E4
:103EA000B9010E946E4F9B01AC01C501B4010E9493
:103EB0004E5003C060E070E0CB010E9434500E947D
:103EC000B6502B013C016D817E818F819885909544
:103ED0008095709561957F4F8F4F9F4F0E94E9505D
:103EE0004B015C01F101E05CFF4F608171818281D7
:103EF00093810E94E7506D837E838F83988720E0B3
:103F000030E0A901C501B4010E944750882349F15E
:103F10002D813E814F815885CA01B9010E941C53F1
:103F20006D8B7E8B8F8B988FA7019601C701B60191
:103F30000E941C539B01AC016D897E898F89988DED
:103F40000E946D4F6B017C01A5019401C501B40174
:103F50000E946E4F9B01AC01C701B6010E944E50FA
:103F600003C060E070E0CB010E942451D101509663
:103F70008D909D90AD90BC90539775016401C418CD
:103F8000D508E608F7080E94B650C61AD70AE80A0C
:103F9000F90AF7FE6BC020E030E0A90169817A815F
:103FA0008B819C810E944750882309F447C0298156
:103FB0003A814B815C81CA01B9010E946E4F6B014D
:103FC0007C01C501B4010E94E7509B01AC01C7010F
:103FD000B6010E941C536B017C0129853A854B85F3
:103FE0005C85CA01B9010E941C539B01AC01C70149
:103FF000B6010E946D4F6B017C012D813E814F8186
:104000005885CA01B9010E941C539B01AC01C7012C
:10401000B6010E946E4F6B017C0120E030E040E869
:1040200050E469817A818B819C810E941C539B01A1
:10403000AC01C701B6010E944E5003C060E070E0C1
:10404000CB010E9434500E94B6502B013C0197FFD7
:1040500003C0412C512C3201481459046A047B04DA
:1040600010F024013501C12CD12C76018FB7F894C2
:10407000F101E45BFF4F9081911121C0F101448A6D
:10408000558A668A778AC40CD51CE61CF71CD101B8
:10409000C08ED18EE28EF38E2D853E854F85588958
:1040A00024AF35AF46AF57AFA05CBF4F29893A89DF
:1040B0004B895C892D933D934D935C9313978FBFF0
:1040C00068960FB6F894DEBF0FBECDBFDF91CF91DB
:1040D0001F910F91FF90EF90DF90CF90BF90AF9026
:1040E0009F908F907F906F905F904F903F902F9018
:1040F00008954F925F926F927F92AF92BF92CF924C
:10410000DF92EF92FF920F931F93CF93DF93EB0118
:104110007A01209709F458C04115510509F454C09B
:10412000AAA4BBA40CA51DA59501A8016EA17FA101
:1041300088A599A50E944750882309F445C08FA9F6
:1041400081113AC0F70146A057A060A471A4A30151
:104150009201B501C8010E944A5218166CF5A301DC
:104160009201C301B2010E941C536B017C018AA918
:104170009BA9ACA9BDA9BC01CD0190589B01AC0184
:104180000E946E4F2EA53FA548A959A90E941C5315
:104190009B01AC01C701B6010E946D4F0E9489537B
:1041A0006B017C019B01AC01B501C8010E94475025
:1041B00087FD02C056018701A501B8014EA35FA388
:1041C00068A779A781E08EABDF91CF911F910F9106
:1041D000FF90EF90DF90CF90BF90AF907F906F9067
:1041E0005F904F900895DF92EF92FF920F931F938D
:1041F000CF93DF93809179048FB7F894E09078049F
:104200008FBF8091790490E08E1991098F70992762
:104210000497F4F01091790413501F7040E050E0BF
:1042200000E0F12C8DE4D82E1E1591F0111101C083
:1042300010E11150D19EE0011124C658DB4F602FD0
:104240007F2DCE0156DF402F5F2D0C2FFD2EECCFA2
:10425000DF91CF911F910F91FF90EF90DF90089524
:104260004F925F926F927F92AF92BF92CF92DF9206
:10427000EF92FF920F931F93CF93DF938C01EB018B
:10428000009709F453C0FC0187A981114FC046A0D3
:1042900057A060A471A4AEA0BFA0C8A4D9A49501E2
:1042A000A601C301B2010E94475087FF3FC0A3018E
:1042B0009201C301B2010E941C532B013C01F80181
:1042C00082A993A9A4A9B5A9BC01CD0190589B01CD
:1042D000AC010E946E4FF80126A537A540A951A94F
:1042E0000E941C539B01AC01C301B2010E946D4F9F
:1042F0000E9489537B018C019B01AC01B501C60171
:104300000E94475087FF02C0750186019701A801EE
:10431000B501C6010E944750882341F0A701B801AA
:104320004EA35FA368A779A781E08EABDF91CF9101
:104330001F910F91FF90EF90DF90CF90BF90AF90C3
:104340007F906F905F904F900895EF92FF920F9340
:104350001F93CF93DF93F090780400E010E080E0AB
:1043600090E02DE4E22E20917904F21689F0EF9C82
:10437000E0011124C658DB4FAE01B80171DF81E0C6
:104380008F0D803109F480E0F82EC8018E01EBCF4B
:1043900040E050E0B801DF91CF911F910F91FF9065
:1043A000EF905ECF4F925F926F927F928F929F922B
:1043B000AF92BF92CF92DF92EF92FF920F931F9333
:1043C000CF93DF9390907804C0E0D0E03DE4832E5B
:1043D000892D992787FD90952091790430E08217E7
:1043E0009307B9F1889E5001899EB00C1124C50134
:1043F00086589B4F5C01209729F18EA9811104C03A
:10440000F50186A98823F1F0CAA0DBA0ECA0FDA0ED
:10441000A7019601F50166A177A180A591A50E944B
:104420004E502B013C01A70196016EA17FA188A5EA
:1044300099A50E944E50AB01BC0193018201CE01AF
:1044400081DC1EAA9394F0E19F1201C0912CE5013A
:10445000BFCF2097E9F0CAA0DBA0ECA0FDA0A70188
:1044600096016DEC7CEC8CE49DE30E944E504B0178
:104470005C01A70196016EA17FA188A599A50E9464
:104480004E50AB01BC0195018401CE015BDC1EAA3C
:10449000DF91CF911F910F91FF90EF90DF90CF9020
:1044A000BF90AF909F908F907F906F905F904F9054
:1044B000089599DE4ADF76CF10927904109278043D
:1044C00080E1EFE5F9E0DF011D928A95E9F71092AE
:1044D0004F091092500910925109109252091092EE
:1044E00053091092540910925509109256091092CE
:1044F0005709109258091092590910925A091092AE
:104500005B0910925C0910925D0910925E0910928D
:104510004B0910924C0910924D0910924E090895C2
:104520004F925F926F927F928F929F92AF92BF92C3
:10453000CF92DF92EF92FF920F931F93CF93DF936F
:1045400080914A09882309F4EFC0C0901E02D090E0
:104550001F02E0902002F0902102609128047091E7
:104560002904882777FD8095982F0E94E95020E044
:1045700030E040E050E40E946E4F9601A7010E9497
:10458000475087FDD1C050907804612C712C00E019
:1045900010E04DE4442E80917904581609F453C07C
:1045A000852D90E0489EF001499EF00D1124E658BB
:1045B000FB4F4081518162817381452B462B472BF4
:1045C00081F44481558166817781452B462B472BA9
:1045D00041F44085518562857385452B462B472BD9
:1045E00069F1489EE001499ED00D1124C658DB4F69
:1045F0006C857D858E859F850E94E9504B015C010D
:10460000688979898A899B890E94E7509B01AC015E
:10461000C501B4010E944E502AA13BA14CA15DA14D
:104620000E941C535B01D82FC92F9301A8010E943F
:104630004A5218161CF435010D2F1C2F5394852D4A
:104640008F70582EA8CF20911A0230911B024091F2
:104650001C0250911D02B301C8010E941C539B0112
:10466000AC01B601C7010E946E4F8B01D82FC92F34
:104670009601A7010E94475087FD03C06801ED2EF7
:10468000FC2E0091220210912302D0912402C091AD
:10469000250298014D2F5C2FB601C7010E944A5296
:1046A00018161CF08601DE2DCF2D8090730490909B
:1046B0007404A0907504B090760498014D2F5C2F7F
:1046C000C501B4010E944A521816D4F420E037ED17
:1046D00043EA5CE3B8018D2F9C2F0E941C536B01B1
:1046E0007C0128E431EE4AE75FE3C501B4010E9492
:1046F0001C53A70196010E946E4F8B01D82FC92F22
:10470000C801AD2FBC2F8093730490937404A093C1
:104710007504B0937604B8018D2F9C2F0E94B6507B
:104720007093290460932804DF91CF911F910F911A
:10473000FF90EF90DF90CF90BF90AF909F908F90C1
:104740007F906F905F904F9008956091A20B909131
:10475000780480917904981781F0809178049DE421
:10476000899FF0011124EE53FB4F608190917904F1
:10477000891719F08F5F8F70F9CF70E088E00E9481
:10478000A94ECECE2F923F924F925F926F927F9220
:104790008F929F92AF92BF92CF92DF92EF92FF9251
:1047A0000F931F93CF93DF93CDB7DEB7CC56D109CC
:1047B0000FB6F894DEBF0FBECDBF2C015B014A01DE
:1047C0003901E8A6F8AE25960FAF25971CAF8601F4
:1047D000209179042F5F29962FAF2997203119F462
:1047E00029961FAE299729963FAD2997E32EFF24DE
:1047F000E7FCF0948091780490E08E159F0529F4F1
:104800000E94340B0E942F3AF5CF2091AB093091D2
:10481000AC094091AD095091AE09D2016D917D91E5
:104820008D919C910E941C530E94EC5269966CAF32
:104830007DAF8EAF9FAF69972091AF093091B009DE
:104840004091B1095091B209F50160817181828175
:1048500093810E941C530E94EC526D966CAF7DAF09
:104860008EAF9FAF6D972091B3093091B4094091FD
:10487000B5095091B609D4016D917D918D919C91AE
:104880000E941C530E94EC52A1966CAF7DAF8EAF7C
:104890009FAFA1972091B7093091B8094091B9090C
:1048A0005091BA09F30160817181828193810E94E4
:1048B0001C530E94EC5224966CAF7DAF8EAF9FAF1D
:1048C000249780916B0990916C09A0916D09B0912A
:1048D0006E0924962CAD3DAD4EAD5FAD24972817E3
:1048E00039074A075B0709F497C0E091A40B34E04D
:1048F000E39FF0011124E05EFB4F20E030E040EF49
:1049000052E460817181828193810E94475087FFC8
:104910001DC080917704811119C00C940A2D9091CB
:10492000C00095FFFCCF8093C60031968491811121
:10493000F6CFEFE5FDE0849181110C941C2D809160
:10494000C00085FFFCCF8AE08093C60080916B0990
:1049500090916C09A0916D09B0916E0924962CADCF
:104960003DAD4EAD5FAD2497281B390B4A0B5B0B59
:10497000CA01B90157FF07C0909580957095619560
:104980007F4F8F4F9F4F0E94E9506B017C0120E0C9
:1049900030E44FE054E46091B7097091B809809118
:1049A000B9099091BA090E941C539B01AC01C7013F
:1049B000B6010E944A5218167CF524968CAD9DAD26
:1049C000AEADBFAD249780936B0990936C09A09313
:1049D0006D09B0936E09E9E7FDE08491882341F009
:1049E0009091C00095FFFCCF8093C6003196F5CF23
:1049F000E1E4FDE08491882341F09091C00095FFAF
:104A0000FCCF8093C6003196F5CF8091C00085FF22
:104A1000FCCF8AE08093C600809179049DE4899F51
:104A200010011124D101A658BB4F1D01FD01E45B0B
:104A3000FF4F108220915F09309160094091610918
:104A4000509162092BA33CA34DA35EA369964CAC85
:104A50005DAC6EAC7FAC6997421A530A640A750A62
:104A600077FE08C07094609450944094411C511C8F
:104A7000611C711CD1014D925D926D927C921397D5
:104A8000209163093091640940916509509166094C
:104A90002CAB3DAB4EAB5FAB6D968CAC9DACAEAC76
:104AA000BFAC6D97821A930AA40AB50AB7FE08C074
:104AB000B094A09490948094811C911CA11CB11C72
:104AC000D10114968D929D92AD92BC921797209130
:104AD0006709309168094091690950916A092CA7CA
:104AE0003DA74EA75FA7A196CCACDDACEEACFFAC6A
:104AF000A197C21AD30AE40AF50AF7FE08C0F09497
:104B0000E094D094C094C11CD11CE11CF11CD101D3
:104B10001896CD92DD92ED92FC921B9720916B0935
:104B200030916C0940916D0950916E0928AB39ABF9
:104B30004AAB5BAB24962CAD3DAD4EAD5FAD24973B
:104B400088A999A9AAA9BBA9281B390B4A0B5B0BF9
:104B500057FF07C050954095309521953F4F4F4FD7
:104B60005F4FA0913B02B0913C020E94E25324E6C9
:104B700030E040E050E00E942C54D1011C962D936F
:104B80003D934D935C931F97C814D904EA04FB042A
:104B900014F475016401C216D306E406F50614F494
:104BA00069017A01D301C2014C145D046E047F04D3
:104BB00014F4D701C601F101808B918BA28BB38BCA
:104BC0000697A105B10508F440C7E85BFF4F809147
:104BD000A20B9091A30BAA2797FDA095BA2F8083D3
:104BE0009183A283B38369962CAD3DAD4EAD5FAD8D
:104BF00069978BA19CA1ADA1BEA1281739074A07CF
:104C00005B0724F0D10190961C9203C081E0F10172
:104C100080A36D962CAD3DAD4EAD5FAD6D978CA96B
:104C20009DA9AEA9BFA9281739074A075B073CF41D
:104C3000D10190968C919097826090968C93A196DA
:104C40002CAD3DAD4EAD5FADA1978CA59DA5AEA59C
:104C5000BFA5281739074A075B073CF4D101909696
:104C60008C919097846090968C9324962CAD3DAD5A
:104C70004EAD5FAD249788A999A9AAA9BBA9281709
:104C800039074A075B073CF4D10190968C919097C5
:104C9000886090968C93F8018081D10191968C93D5
:104CA00045284628472809F01798F1018481958105
:104CB000A681B781892B8A2B8B2B09F01698F101DD
:104CC00080859185A285B385892B8A2B8B2B09F052
:104CD0001598F10184859585A685B785892B8A2B42
:104CE0008B2B09F01498D1011C962D913D914D917B
:104CF0005C911F972D962CAF3DAF4EAF5FAF2D97B8
:104D0000232B242B252B01F5B0917F09BBA3E09128
:104D10008009EFA300918109109182092B2F3E2F6A
:104D2000A80168A578AD25968FAD25979CAD0E940A
:104D3000475087FD16C0F8A5FBA328AD2FA32596E5
:104D40000FAD25971CAD0DC0309197093BA3409145
:104D500098094FA30091990910919A09232F342F94
:104D6000DFCF80915F0990916009A0916109B091B6
:104D7000620969962CAD3DAD4EAD5FAD6997281BBC
:104D8000390B4A0B5B0BCA01B9010E94E950209113
:104D9000AB093091AC094091AD095091AE090E9428
:104DA0004E5068A779A78AA79BA7698B7A8B8B8BB4
:104DB0009C8B6D966CAD7DAD8EAD9FAD6D972CA926
:104DC0003DA94EA95FA9621B730B840B950B0E9432
:104DD000E9502091AF093091B0094091B10950914B
:104DE000B2090E944E504B015C016D8B7E8B8F8B04
:104DF000988FA1966CAD7DAD8EAD9FADA1972CA582
:104E00003DA54EA55FA5621B730B840B950B0E94FD
:104E1000E9502091B3093091B4094091B5095091FE
:104E2000B6090E944E506B017C01698F7A8F8B8F7F
:104E30009C8F24966CAD7DAD8EAD9FAD249728A937
:104E400039A94AA95BA9621B730B840B950B0E94BD
:104E5000E9502091B7093091B8094091B9095091B2
:104E6000BA090E944E502B013C0160913B027091A7
:104E70003C02882777FD8095982F0E94E9509B017E
:104E8000AC01C301B2010E941C5320E030E048ECA9
:104E900052E40E944E506D8F7E8F8F8F98A3D10168
:104EA0002D913D914D915C91139728AF39AF4AAF49
:104EB0005BAF263031054105510504F514964D9040
:104EC0005D906D907C901797B6E04B16510461048D
:104ED0007104A4F4F1014084518462847384F6E087
:104EE0004F165104610471044CF4DC01CB01BF770F
:104EF000F10186A797A7A0ABB1AB27C068A579A59C
:104F00008AA59BA50E94C7532B013C01C501B40192
:104F10000E94C7539B01AC01C301B2010E946E4FB6
:104F20004B015C01C701B6010E94C7539B01AC0154
:104F3000C501B4010E946E4F0E948953D1019E9613
:104F40006D937D938D939C93D197D1019E962D91D6
:104F50003D914D915C91D19728962CAF3DAF4EAFCE
:104F60005FAF289760E070E080E89FE30E944E50BA
:104F70009B01AC016BA17FA1C8010E941C532B01B6
:104F80003C019091790480917804E92FF0E0E81BCE
:104F9000F109EF70FF27FDABECABA301920160E0DC
:104FA00074E284E799E40E944E500E94EC526B0137
:104FB0007C012CA93DA9223031050CF442C04901E5
:104FC000AA2497FCA094BA2CC501B4010E94E95010
:104FD00020E030E040E051E40E94475087FF31C0BC
:104FE0008091CB099091CC09A091CD09B091CE09C7
:104FF000C816D906EA06FB0620F5BC01CD016C19DE
:105000007D098E099F09660F771F881F991FA501CB
:1050100094010E940A54CA01B9010E94E7500E94FB
:10502000EC526C0D7D1D8E1D9F1D0E94E7509B0153
:10503000AC0160E074E284E799E40E944E502B01D9
:105040003C01A301920128966CAD7DAD8EAD9FAD64
:1050500028970E941C536CAF7DAF8EAF9FAFD101DC
:1050600092966D937D938D939C93959750966D91A9
:105070007D918D919C9153970E94E7506BA37CA3E7
:105080008DA39EA3A30192010E941C530E94345041
:105090000E94BB506B017C01F10160AF71AF82AF28
:1050A00093AF8E010F5E1F4F2BEB39E065963FAF3C
:1050B0002EAF6597AE014F5D5F4F5AA349A3CE0156
:1050C000019663969FAF8EAF63971FA21CA690E8D0
:1050D00098ABAFE3A8A7F80161917191819191918B
:1050E0008F01A30192010E941C536396AEADBFAD28
:1050F00063976D937D938D939D936396BFAFAEAF92
:1051000063979B01AC015F7761962CAF3DAF4EAFCB
:105110005FAF61976596AEADBFAD65978D909D9081
:10512000AD90BD906596BFAFAEAF6597A5019401F8
:1051300061966CAD7DAD8EAD9FAD61970E944A5278
:105140001816F4F461962CAD3DAD4EAD5FAD619790
:10515000C501B4010E944E50B62EA72E982E892E5E
:10516000262F372F482F592F6FA17CA588A998A5E6
:105170000E94475087FD04C0BFA2ACA698AA88A68B
:10518000E9A1FAA10E171F0709F0A5CF20E030E032
:1051900040E85FE36FA17CA588A998A50E944750CD
:1051A00087FF3DC05E01F1E1AF0EB11C8E010F5FC4
:1051B0001F4F2FA13CA548A958A5D8016D917D91FD
:1051C0008D919C910E941C53F8016193719381937E
:1051D00091938F01EA15FB0561F72FA13CA548A922
:1051E00058A56CAD7DAD8EAD9FAD0E941C53D10115
:1051F00092966D937D938D939C939597C701B6017D
:105200000E94E7502FA13CA548A958A50E941C5315
:105210000E94BB50F10160AF71AF82AF93AF28968F
:105220002CAD3DAD4EAD5FAD28976BA17CA18DA19E
:105230009EA10E944E506B017C0128AD39AD4AAD54
:105240005BAD232B242B252B59F5F101848195810E
:10525000A681B781892B8A2B8B2B11F580859185AF
:10526000A285B385892B8A2B8B2BD1F420918F09B2
:10527000309190094091910950919209C701B6016E
:105280000E941C530E94345081010C5B1F4F0E94EE
:10529000BB50D8016D937D938D939C931397F6C06B
:1052A0002091930930919409409195095091960964
:1052B000C701B6010E941C530E9434500E94BB508B
:1052C00081010C5B1F4FF80160837183828393839C
:1052D00040906F0950907009609071097090720948
:1052E0000E94E7504B015C0168AD79AD8AAD9BAD82
:1052F0000E94E9509B01AC01C501B4010E941C53FE
:105300002BA13CA14DA15EA10E944E504B015C011E
:10531000C301B2010E94E7509B01AC01C501B40179
:105320000E944A52181634F4D8014D925D926D9243
:105330007C9213974090730950907409609075099E
:1053400070907609F80160817181828193810E9459
:10535000E7504B015C01D10114966D917D918D91C7
:105360009C9117970E94E9509B01AC01C501B401C3
:105370000E941C532BA13CA14DA15EA10E944E5046
:105380004B015C01C301B2010E94E7509B01AC01DB
:10539000C501B4010E944A5218162CF4F80140824B
:1053A00051826282738240907B0950907C096090A8
:1053B0007D0970907E0981010C5B1F4FD8016D91B2
:1053C0007D918D919C910E94E7504B015C012D963F
:1053D0006CAD7DAD8EAD9FAD2D970E94E9509B01C8
:1053E000AC01C501B4010E941C532BA13CA14DA1ED
:1053F0005EA10E944E504B015C01C301B2010E94AC
:10540000E7509B01AC01C501B4010E944A52181635
:105410002CF4F801408251826282738240907709B5
:10542000509078096090790970907A09D8016D914F
:105430007D918D919C910E94E7504B015C01F1019F
:1054400060857185828593850E94E9509B01AC013E
:10545000C501B4010E941C532BA13CA14DA15EA12A
:105460000E944E504B015C01C301B2010E94E75003
:105470009B01AC01C501B4010E944A52181634F4D4
:10548000D8014D925D926D927C921397F101EC5B85
:10549000FF4F60817181828193810E94E7504B01AF
:1054A0005C01A70196010E944E50A5966CAF7DAF9E
:1054B0008EAF9FAFA597F10162AB73AB84AB95AB99
:1054C0002DEB37E346E051E4C501B4010E941C53C3
:1054D0000E94B650D1015C966D937D938D939C9301
:1054E0005F97C0908B09D0908C09E0908D09F09067
:1054F0008E0920E030E040E05FE3C701B6010E9482
:105500001C536BA37FA38C0129853A854B855C8551
:10551000A9962CAF3DAF4EAF5FAFA9978091870999
:1055200090918809A0918909B0918A098CAF9DAFAB
:10553000AEAFBFAF20E030E040E05FE3BC01CD01A3
:105540000E941C53B62EA72E982E892EA9966CADBC
:105550007DAD8EAD9FADA9979F772B2D3A2D492D0F
:10556000582D0E944A5218167CF42B2D3A2D492DA5
:10557000582D6BA17FA1C8010E94475087FD04C030
:10558000BBA2AFA2092D182D2D853E854F855889C8
:10559000AD962CAF3DAF4EAF5FAFAD978091830915
:1055A00090918409A0918509B09186092D968CAFC0
:1055B0009DAFAEAFBFAF2D9720E030E040E05FE39E
:1055C000BC01CD010E941C53B62EA72E982E892E09
:1055D000AD966CAD7DAD8EAD9FADAD979F772B2D0C
:1055E0003A2D492D582D0E944A5218167CF42B2D25
:1055F0003A2D492D582D6BA17FA1C8010E9447501B
:1056000087FD04C0BBA2AFA2092D182DD10192962F
:10561000BC91BCA7F101F3A1F8ABD1019496BC9168
:10562000B8A7F101F5A1F8AF2CA538A94B2F5F2F32
:105630006BA17FA1C8010E94475087FD06C02CA521
:105640002BA338A93FA308A518AD4CA95DA94230EA
:1056500051050CF405C150914B095CAB80914C098C
:105660002E968FAF2E9790914D0962969FAF6297BD
:10567000A0914E096496AFAF649727E137EB41EDF7
:1056800058E36CA9782F892F9A2F0E944A52181636
:105690000CF0E6C020914F0930915009409151091A
:1056A0005091520969817A818B819C810E946D4F52
:1056B0002B013C0120915309309154094091550927
:1056C000509156096D817E818F8198850E946D4F22
:1056D0004B015C01A3019201C301B2010E941C5362
:1056E0002B013C01A5019401C501B4010E941C538A
:1056F0009B01AC01C301B2010E946E4F0E9489530D
:105700004B015C01A70196010E944A5218164CF405
:10571000A5019401C701B6010E944E505B014C01E6
:1057200006C0A12CB12C50E8852E6FE3962E209157
:105730005709309158094091590950915A09A99631
:105740006CAD7DAD8EAD9FADA9970E946D4F6B0185
:105750007C01E894F7F82CAD3DAD4EAD5FADC701CF
:10576000B6010E944A521816D4F4A70196016CADF6
:105770007DAD8EAD9FAD0E944E50F62EE72ED82EF9
:10578000C92E262F372F482F592FB501C4010E944B
:10579000475087FD04C0AF2CBE2C8D2C9C2C209133
:1057A0005B0930915C0940915D0950915E09AD96AD
:1057B0006CAD7DAD8EAD9FADAD970E946D4F6B0111
:1057C0007C01E894F7F82D962CAD3DAD4EAD5FAD64
:1057D0002D97C701B6010E944A521816E4F4A7019A
:1057E00096012D966CAD7DAD8EAD9FAD2D970E942F
:1057F0004E50F62EE72ED82EC92E262F372F482FA3
:10580000592FB501C4010E94475087FD04C0AF2C39
:10581000BE2C8D2C9C2C9501A4016CA578A988A583
:1058200098AD0E941C534B015C019B01AC016CA91B
:105830002E967FAD2E9762968FAD629764969FAD40
:1058400064970E94475087FF0EC08CA82E969FAC8D
:105850002E976296AFAC62976496BFAC649703C014
:105860008BA09FA05801C401D501F10182A793A785
:10587000A4A7B5A7A5966CAD7DAD8EAD9FADA59740
:1058800090589B01AC010E946E4F28962CAD3DAD07
:105890004EAD5FAD28970E941C539B01AC016BE09D
:1058A00077ED83E29BE30E946D4F0E9489537B0159
:1058B000D82EC92E9B01482F592FB401C5010E9433
:1058C000475087FD03C04701AD2CBC2CC401D50156
:1058D000F10186A397A3A0A7B1A797014D2D5C2D39
:1058E0006CA578A988A598AD0E94475018162CF091
:1058F00081E0D101D7968C9302C0F10117AA81E013
:10590000D101D6968C9380E1FE013196AFE4B9E0E7
:1059100001900D928A95E1F78CA598A9A8A5B8AD3C
:1059200080934B0990934C09A0934D09B0934E0975
:105930009C01AD016BA17FA1C8010E944E506B017B
:105940007C012CA538A948A558ADB401C5010E9419
:105950004E50AB01BC0197018601C1010E94A21EFD
:105960002996BFAD2997B093790469962CAD3DADCA
:105970004EAD5FAD699720935F0930936009409306
:105980006109509362096D968CAD9DADAEADBFAD12
:105990006D978093630990936409A0936509B09310
:1059A0006609A1962CAD3DAD4EAD5FADA19720939C
:1059B0006709309368094093690950936A092496EE
:1059C0008CAD9DADAEADBFAD249780936B09909328
:1059D0006C09A0936D09B0936E090E945922C459B5
:1059E000DF4F0FB6F894DEBF0FBECDBFDF91CF9172
:1059F0001F910F91FF90EF90DF90CF90BF90AF90ED
:105A00009F908F907F906F905F904F903F902F90DE
:105A10000C94A61424962CAD3DAD4EAD5FAD2497ED
:105A200020936B0930936C0940936D0950936E0974
:105A3000E9E7FDE00C9496249091C00095FFFCCF1F
:105A40008093C60031960C949B24C459DF4F0FB647
:105A5000F894DEBF0FBECDBFDF91CF911F910F91A4
:105A6000FF90EF90DF90CF90BF90AF909F908F907E
:105A70007F906F905F904F903F902F900895EF929E
:105A8000FF920F931F93CF93DF937B018A01E9016C
:105A90002091AB093091AC094091AD095091AE090C
:105AA000FC0160817181828193810E941C530E945C
:105AB000EC5260935F097093600980936109909341
:105AC00062092091AF093091B0094091B10950911C
:105AD000B209F70160817181828193810E941C5318
:105AE0000E94EC5260936309709364098093650986
:105AF000909366092091B3093091B4094091B5099A
:105B00005091B609F80160817181828193810E9470
:105B10001C530E94EC52609367097093680980934C
:105B2000690990936A092091B7093091B8094091A9
:105B3000B9095091BA09688179818A819B810E9453
:105B40001C530E94EC5260936B0970936C09809314
:105B50006D0990936E092BE639E047E659E063E65C
:105B600079E08FE599E00E94F51B10924B091092A5
:105B70004C0910924D0910924E0910924F09109243
:105B80005009109251091092520910925309109223
:105B90005409109255091092560910925709109203
:105BA00058091092590910925A0910925B091092E3
:105BB0005C0910925D0910925E09DF91CF911F91EF
:105BC0000F91FF90EF9008952091B7093091B80997
:105BD0004091B9095091BA09FC01608171818281BB
:105BE00093810E941C530E94EC5260936B09709346
:105BF0006C0980936D0990936E098BE699E00C9483
:105C0000311C8093770408952F923F924F925F92B8
:105C10006F927F928F929F92AF92BF92CF92DF92BC
:105C2000EF92FF920F931F93CF93DF93CDB7DEB721
:105C3000C454D1090FB6F894DEBF0FBECDBF3C01EE
:105C40001B014A012FA309A7EBA62196ACAEBDAE5E
:105C5000CEAEDFAE219734E0239F20011124440D06
:105C6000551D5AAB49ABDA01CD90DD90ED90FC901B
:105C7000FC01E40DF51D2081318142815381C70172
:105C8000B6010E946E4F6BAB7CAB8DAB9EABB4E0AC
:105C90000B9F80011124F401E00FF11FF8AFEFAB6F
:105CA00080809180A280B380F301E00FF11F2081FA
:105CB000318142815381C501B4010E946E4F69AFA9
:105CC0007AAF8BAF9CAF2BA5F4E02F9FC0011124BE
:105CD000F301E80FF91F2081318142815381298F1F
:105CE0003A8F4B8F5C8FF101E80FF91F6081718152
:105CF000828193810E946D4F6F8F78A389A39AA3AD
:105D0000D1011C968D919D910D90BC91A02D8DA7D8
:105D10009EA7AFA7B8ABD3011C962D913D914D9195
:105D20005C911F972BA33CA34DA35EA3A7019601F3
:105D300050582D8B3E8B4F8B588FD501C401B058D6
:105D4000898B9A8BAB8BBC8BF101E40DF51D2BA9D4
:105D50003CA94DA95EA960817181828193810E94D5
:105D60006D4F6B017C01F101E00FF11F29AD3AADE0
:105D70004BAD5CAD60817181828193810E946D4FDA
:105D80004B015C01A70196016D897E898F89988DF1
:105D90000E941C532B013C01A501940169897A8959
:105DA0008B899C890E941C539B01AC01C301B201E9
:105DB0000E946E4F2B013C01A50194016D897E89E3
:105DC0008F89988D0E941C534B015C01A70196019D
:105DD00069897A898B899C890E941C539B01AC013B
:105DE000C501B4010E946D4FA30192010E94E14FD1
:105DF0006B017C0120E030E0A9010E94475087FF41
:105E00000AC02BED3FE049EC50E4C701B6010E9407
:105E10006E4F6B017C016F968FAD6F97882351F0A9
:105E20002BED3FE049EC50E4C701B6010E946D4FF5
:105E30006B017C016E962CAD3DAD4EAD5FAD6E97A6
:105E4000C701B6010E941C532F8D38A149A15AA148
:105E50005F770E9457524B015C012FE632E143E825
:105E60005AE30E94475087FDC5C1C501B4010E9495
:105E700024510E94BB507E8F6D8FDB01AB2B21F430
:105E8000E1E0F0E0FE8FED8F2D8D3E8DB90180E0D9
:105E900090E00E94E7504B015C019B01AC01C701FF
:105EA000B6010E944E502B013C01A50194016F8D5B
:105EB00078A189A19AA10E944E5025966CAF7DAF22
:105EC0008EAF9FAF25972BA13CA14DA15EA16DA5E3
:105ED0007EA58FA598A90E946D4FA50194010E94EF
:105EE0004E506DA77EA78FA798AB20E030E040E032
:105EF0005FE3C301B2010E941C53A30192010E94FF
:105F00001C539B01AC0160E070E080E89FE30E94BD
:105F10006D4F6F8F78A389A39AA3CE010196FC01E0
:105F20004BA534E0439FE00DF11D1124298D3A8DDE
:105F30004B8D5C8D20833183428353832BA13CA105
:105F40004DA15EA12D873E874F87588BB12C41E034
:105F500050E05A8F498F81E090E08C0F9D1FBFA1C8
:105F6000A4E0BA9F800D911D11249CA78BA721E06E
:105F700030E02C0F3D1F59A544E0549F200D311DEA
:105F800011243AA729A7F8A7EFA3498D5A8D8D8D23
:105F90009E8D4817590708F017C188E18B150CF43E
:105FA00044C02F8D38A149A15AA169897A898B896A
:105FB0009C890E941C536B017C01A30192016D8995
:105FC0007E898F89988D0E941C53A70196010E949B
:105FD0006E4FA62E172F982E892E2F8D38A149A1EE
:105FE0005AA16D897E898F89988D0E941C536B01FF
:105FF0007C01A301920169897A898B899C890E941D
:106000001C539B01AC01C701B6010E946D4F6D8B03
:106010007E8B8F8B988FB3948A2D912FA92DB82DBD
:10602000898B9A8BAB8BBC8B6AC0A98DBA8DBD0155
:1060300080E090E00E94E750A30192010E941C536F
:106040006B017C010E944B50698B7A8B8B8B9C8BF4
:10605000C701B6010E947F534B015C01E9A9FAA96F
:10606000C080D180E280F380F7FAF094F7F8F094E2
:10607000AFA9B8AD2D913D914D915C912BA33CA35F
:106080004DA35EA329893A894B895C89C701B60172
:106090000E941C536D8B7E8B8F8B988FA501940172
:1060A0006BA17CA18DA19EA10E941C539B01AC0100
:1060B0006D897E898F89988D0E946E4F6D8B7E8B46
:1060C0008F8B988FA5019401C701B6010E941C53C4
:1060D0006B017C0129893A894B895C896BA17CA180
:1060E0008DA19EA10E941C539B01AC01C701B6016A
:1060F0000E946D4F698B7A8B8B8B9C8BB12C2D8979
:106100003E894F89588D6BA97CA98DA99EA90E94B3
:106110006E4FEBA5FCA560837183828393832989ED
:106120003A894B895C8969AD7AAD8BAD9CAD0E9493
:106130006E4FA9A5BAA56D937D938D939C931397EC
:1061400025962CAD3DAD4EAD5FAD2597EFA1F8A5E1
:1061500060817181828193810E946E4FAFA1B8A549
:106160006D937D938D939C9313972DA53EA54FA57D
:1061700058A96D857E858F8598890E946E4F6D87A1
:106180007E878F87988BCE01019639D7FE01E15A21
:10619000FF4F6F012196ECACFDAC0EAD1FAD21970A
:1061A0009E01235F3F4FAE01475F5F4FBE016B5FB4
:1061B0007F4FCE0101960E94C223298D3A8D2F5F19
:1061C0003F4F3A8F298FE1CE9101245F3F4FA101CC
:1061D000485F5F4FB1016C5F7F4FDE01A15ABF4F37
:1061E0006D012196ECACFDAC0EAD1FAD2197C10148
:1061F0000E94C223CC5BDF4F0FB6F894DEBF0FBE08
:10620000CDBFDF91CF911F910F91FF90EF90DF9065
:10621000CF90BF90AF909F908F907F906F905F9046
:106220004F903F902F900895FC0165917591859155
:10623000949108952F923F924F925F926F927F9226
:106240008F929F92AF92BF92CF92DF92EF92FF9286
:106250000F931F93CF93DF9300D000D0CDB7DEB75D
:106260008C019C01220F331F220F331F3E832D838D
:106270002354344F3A832983F90110821182128208
:10628000138229EC3BE045EC5BE061EC7BE08DEBBD
:106290009BE0F5DB8D819E81895A9E4EC5DFF8011A
:1062A000E85BFE4E84902D813E812E56344F1901BD
:1062B00020E030E040EC5FE30E941C536B017C0166
:1062C000992487FC9094A92CB92CC501B4010E9493
:1062D000E9509B01AC01C701B6010E941C53F101BA
:1062E00060837183828393832D813E81215C3D4F46
:1062F0003C832B83F901608171818281938160935A
:106300002A0270932B0280932C0290932D0220E09E
:1063100030E040E752E40E944E5024EAC22E2BE0C7
:10632000D22E7B018C012EE93BE04AE95BE066E975
:106330007BE082E99BE00E94C2230E94E91BE98185
:10634000FA81108211821282138229EC3BE045EC23
:106350005BE061EC7BE08DEB9BE091DB8D819E81CE
:10636000855B9E4E61DF2B013C016B017C01F7FADE
:10637000F094F7F8F094C501B4010E94E9509B0134
:10638000AC01C701B6010E941C53F1016083718307
:106390008283938320E030E040E752E460912A0258
:1063A00070912B0280912C0290912D020E944E50F0
:1063B00034EAC32E3BE0D32E7B018C012EE93BE077
:1063C0004AE95BE066E97BE082E99BE00E94C22348
:1063D0000E94E91BA3019201C301B2010E946E4F0A
:1063E0006B017C01C501B4010E94E9509B01AC0125
:1063F000C701B6010E941C53F1016083718382833F
:10640000938320E030E040E05FE3EB81FC8160813A
:106410007181828193810E941C5360932A02709340
:106420002B0280932C0290932D0220E030E040E775
:1064300052E40E944E5044EAC42E4BE0D42E7B011D
:106440008C012EE93BE04AE95BE066E97BE082E90A
:106450009BE00E94C2230E94E91B8D819E818D5981
:106460009E4EE2DEED81FE81EF54F44FC080D1807C
:10647000E280F380A70196010E946E4F4B015C0100
:10648000E981FA8160837183828393838D819E8108
:1064900085589E4EC9DE0D811E810B55144FA701F4
:1064A00096010E946E4FF80160837183828393830B
:1064B0008D819E8181599E4EB7DE0D811E81015DC9
:1064C0001D4FA70196010E946E4FF80160837183F2
:1064D00082839383F10180829182A282B38210929F
:1064E0002A0210922B0210922C0210922D02269654
:1064F0000FB6F894DEBF0FBECDBFDF91CF911F91D5
:106500000F91FF90EF90DF90CF90BF90AF909F9052
:106510008F907F906F905F904F903F902F900C9452
:106520009C14FC012491222341F03091C00035FFDE
:10653000FCCF2093C6000196F4CF22E030E083ED3B
:106540009BE00C94994BCF93DF931F921F92CDB792
:10655000DEB78091610C9091620C9E012F5F3F4FDE
:10656000009719F427563C4002C0281B390B3A8388
:10657000298389819A810F900F90DF91CF9108959F
:106580009D9AA5980895CF92DF92EF92FF920F9374
:106590001F93CF93DF9300D01F92CDB7DEB7F0DF0C
:1065A00040E052EC61E070E083ED9BE00E94B9496D
:1065B000E2E4F1E18491882341F09091C00095FFDD
:1065C000FCCF8093C6003196F5CF8091C00085FF47
:1065D000FCCF8AE08093C60087E891E1FC0124911A
:1065E000222341F03091C00035FFFCCF2093C6003C
:1065F0003196F5CF24B720FF14C0EAE3F1E13491DE
:10660000332341F04091C00045FFFCCF3093C600DA
:106610003196F5CF3091C00035FFFCCF3AE0309392
:10662000C60021FF14C0EAE2F1E13491332341F0C6
:106630004091C00045FFFCCF3093C6003196F5CFA6
:106640003091C00035FFFCCF3AE03093C60022FF06
:1066500014C0E9E1F1E13491332341F04091C000ED
:1066600045FFFCCF3093C6003196F5CF3091C00086
:1066700035FFFCCF3AE03093C60023FF14C0E9E0B9
:10668000F1E13491332341F04091C00045FFFCCF4C
:106690003093C6003196F5CF3091C00035FFFCCF66
:1066A0003AE03093C60025FF14C0E9EFF0E12491F1
:1066B000222341F03091C00035FFFCCF2093C6006B
:1066C0003196F5CF2091C00025FFFCCF2AE0209322
:1066D000C60014BEE1EFF0E12491222341F0309195
:1066E000C00035FFFCCF2093C6003196F5CFEBEE0E
:1066F000F0E12491222341F03091C00035FFFCCF1E
:106700002093C6003196F5CF2091C00025FFFCCF25
:106710002AE02093C600FC012491E7E8F1E122235E
:1067200049F03091C00035FFFCCF2093C600319670
:106730002491F5CFEBEDF0E12491222341F030914B
:10674000C00035FFFCCF2093C6003196F5CFE0EDB9
:10675000F0E12491222341F03091C00035FFFCCFBD
:106760002093C6003196F5CFE4ECF0E1249122238A
:1067700041F03091C00035FFFCCF2093C600319628
:10678000F5CFECEBF0E12491222341F03091C000F1
:1067900035FFFCCF2093C6003196F5CF2091C00085
:1067A00025FFFCCF2AE02093C600E1EBF0E1249125
:1067B000222341F03091C00035FFFCCF2093C6006A
:1067C0003196F5CFE5EAF0E12491222341F03091B2
:1067D000C00035FFFCCF2093C6003196F5CF209145
:1067E000C00025FFFCCF2AE02093C600FC01849165
:1067F000E7E8F1E1882349F09091C00095FFFCCFD4
:106800008093C60031968491F5CFE6E9F0E184915A
:10681000882341F09091C00095FFFCCF8093C60083
:106820003196F5CF90DE4AE050E0BC0183ED9BE06D
:106830000E94CD4AEFE7F0E18491882341F09091E6
:10684000C00095FFFCCF8093C6003196F5CF4AE09B
:1068500050E060ED74E083ED9BE00E94CD4A8091B2
:10686000C00085FFFCCF8AE08093C6001092ED093E
:106870001092EE091092EF091092F0090E949A4BC3
:106880005BE9C52E59E0D52E6BEAE62E69E0F62EBF
:106890000FE619E0F60161917191819191916F017B
:1068A000F70121913191419151917F0129833A83DF
:1068B0004B835C830E94E75029813A814B815C8144
:1068C0000E941C530E94BB50F80161937193819305
:1068D00091938F01FBEACF16F9E0DF06D9F60E940B
:1068E0000B0D0E945C220F900F900F900F90DF9184
:1068F000CF911F910F91FF90EF90DF90CF900C946C
:10690000671D8091E1099091E20960E070E00196D5
:106910000C947B548091E1099091E2094AE050E0A7
:1069200060E070E001960C94EF55682F772767FDC3
:1069300070952091EB093091EC0940E6429FC0012F
:10694000439F900D11248F50964F0E945A57909359
:10695000E2098093E10921E0892B09F420E0822FEC
:1069600008950E940F4D6093DD097093DE098093B6
:10697000DF099093E009E4E1FEE08491882341F08F
:106980009091C00095FFFCCF8093C6003196F5CF63
:106990008091C00085FFFCCF8AE08093C6000895F7
:1069A00083ED9BE00E940B4AE7E1FEE0849188239F
:1069B00041F09091C00095FFFCCF8093C6003196C6
:1069C000F5CF4091760B5091770B6091780B7091D9
:1069D000790B4F5F5F4F6F4F7F4F2AE030E083EDC1
:1069E0009BE00E94AA4A8091C00085FFFCCF8AE00C
:1069F0008093C600B6CF4F925F926F927F928F9234
:106A00009F92AF92BF92CF92DF92EF92FF920F933D
:106A10001F93CF93DF9370E6F72EC4E0D0E0EBE551
:106A2000FFE0D490EAE0EE2EE1EDFFE0C490BB245D
:106A3000B3948091540C9091550C2091560C309148
:106A4000570C821B930B8F779927892B09F419C256
:106A50008091E7099091E80904970CF012C283ED48
:106A60009BE00E94EF498093E6092091E409309170
:106A7000E5098A3061F08D3051F08A3321F490912C
:106A8000E309992321F02F3531050CF41FC121159D
:106A9000310519F41092E309F4C18091E90990914C
:106AA000EA09F89E4001F99E900C1124F401E20FCE
:106AB000F31FEF50F64F10822091E309211101C11D
:106AC0001092E309FC01E351F64F108284010F504C
:106AD000164F6EE470E0C8010E945A570097F1F11A
:106AE0009093E2098093E109801B910B880D991D19
:106AF0004AE050E060E070E08E50964F0E94EF5503
:106B000060937A0B70937B0B80937C0B90937D0B3F
:106B10004090760B5090770B6090780B7090790BCB
:106B20002FEF421A520A620A720A0091E909109183
:106B3000EA09641575058605970509F4E5C0F09E18
:106B4000C001F19E900D11246AE770E18F50964FBD
:106B50000E944057892B09F0D7C066C16AE270E0F5
:106B6000C8010E945A57892B09F444C0EDE8F1E1AD
:106B70008491882341F09091C00095FFFCCF8093D1
:106B8000C6003196F5CFE4EDFFE08491882341F013
:106B90009091C00095FFFCCF8093C6003196F5CF51
:106BA0004091760B5091770B6091780B7091790B37
:106BB0002AE030E083ED9BE00E94AA4A8091C00069
:106BC00085FFFCCF8AE08093C6001092E509109201
:106BD000E40957C180917A0B90917B0BA0917C0BBB
:106BE000B0917D0B8093760B9093770BA093780BED
:106BF000B093790B8091E9099091EA09F89E8001A0
:106C0000F99E100D1124C8018F50964F4C0167E476
:106C100070E00E945A57009709F43EC09093E20931
:106C20008093E10988199909800F911F60E070E055
:106C30008E50964F0E947B540E94B650643071056E
:106C400058F58091CF09811113C08C2DE1EDFFE043
:106C5000882349F09091C00095FFFCCF8093C60037
:106C600031968491F5CF8091C00085FFFCCF12C092
:106C70008D2DEBE5FFE0882349F09091C00095FF52
:106C8000FCCF8093C60031968491F5CF8091C000EF
:106C900085FFFCCFE092C6008091E9099091EA0956
:106CA0000196BE010E94F7539093EA098093E90987
:106CB0008091E7099091E80901969093E809809303
:106CC000E7091092E5091092E409B3CE8B3311F471
:106CD000B092E3099091E3099111ABCE4091E9099B
:106CE0005091EA09B9016F5F7F4F7093E509609396
:106CF000E409F49EF001F59EF00D1124E20FF31F5C
:106D0000EF50F64F808395CEF09E4001F19E900C9F
:106D1000112484010F50164F6AE270E0C8010E94EE
:106D20005A57009789F5EDE8F1E18491882341F005
:106D30009091C00095FFFCCF8093C6003196F5CFAF
:106D4000EEEFFFE08491882341F09091C00095FF21
:106D5000FCCF8093C6003196F5CF4091760B5091D1
:106D6000770B6091780B7091790B2AE030E083ED1E
:106D70009BE00E94AA4A8091C00085FFFCCF8AE078
:106D80008093C6000DDE21CF20E0A12CF401E20F9C
:106D9000F11DEF50F64F30813A3219F02F5FA326E4
:106DA000F5CF9093E2098093E109801B910B880D48
:106DB000991D60E070E08E50964F0E947B540E94B7
:106DC000B6502A2D30E02617370709F403CFEDE837
:106DD000F1E18491882341F09091C00095FFFCCFB0
:106DE0008093C6003196F5CFE8E2F0E184918823E4
:106DF00041F09091C00095FFFCCF8093C600319682
:106E0000F5CF4091760B5091770B6091780B709194
:106E1000790B2AE030E083ED9BE00E94AA4A809142
:106E2000C00085FFFCCFABCFEDE8F1E18491882372
:106E300041F09091C00095FFFCCF8093C600319641
:106E4000F5CFE7E4F0E18491882341F09091C00010
:106E500095FFFCCF8093C6003196F5CF4091760B1D
:106E60005091770B6091780B7091790B2AE030E0AC
:106E700083ED9BE00E94AA4A8091C00085FFFCCF71
:106E80007ECFDF91CF911F910F91FF90EF90DF9018
:106E9000CF90BF90AF909F908F907F906F905F90BA
:106EA0004F9008958F929F92AF92BF92CF92DF92B0
:106EB000EF92FF920F931F93CF93DF93F4EDEF2E9A
:106EC000F3E0FF2E0DEB1BE0C2E9DBE0AFECCA2ED6
:106ED000ABE0DA2EF70181917F0127DD882311F1E4
:106EE00010DD4B015C01F6018081811103C06091CE
:106EF000710B01C061E070E080E090E00E94E95019
:106F0000F80120813181428153810E941C539B01F1
:106F1000AC01C501B4010E946E4F688379838A83F6
:106F20009B8309C0F80180819181A281B38188830C
:106F30009983AA83BB830C5F1F4F2496FFEFCF1A60
:106F4000DF0A88EDE81683E0F80621F686E4EDDC3A
:106F50008823D1F0D6DC6B017C016093820B7093A7
:106F6000830B8093840B9093850B20E030E0A90184
:106F70000E944A52181644F4C0922A02D0922B0260
:106F8000E0922C02F0922D02DF91CF911F910F9190
:106F9000FF90EF90DF90CF90BF90AF909F908F9039
:106FA000089580DF89E4C1DC882351F0AADC609376
:106FB000860B7093870B8093880B9093890B08C086
:106FC0001092860B1092870B1092880B1092890BEF
:106FD0008AE4ABDC882351F094DC60938A0B7093D5
:106FE0008B0B80938C0B90938D0B089510928A0BD2
:106FF00010928B0B10928C0B10928D0B0895CF92E8
:10700000DF92EF92FF92CF93DF93EC01C090A50B3C
:10701000D090A60BE090A70BF090A80BA7019601CB
:10702000688179818A819B810E94475087FF04C0D3
:10703000C882D982EA82FB82C090A90BD090AA0BA9
:10704000E090AB0BF090AC0BA70196016C817D81B9
:107050008E819F810E94475087FF04C0CC82DD82D1
:10706000EE82FF82C090AD0BD090AE0BE090AF0BE4
:10707000F090B00BA7019601688579858A859B857C
:107080000E94475087FF04C0C886D986EA86FB86DF
:10709000C0902F02D0903002E0903102F090320286
:1070A000A7019601688179818A819B810E944A5259
:1070B000181624F4C882D982EA82FB82C090330277
:1070C000D0903402E0903502F0903602A70196018C
:1070D0006C817D818E819F810E944A52181624F412
:1070E000CC82DD82EE82FF82C0903702D0903802DF
:1070F000E0903902F0903A02A701960168857985FF
:107100008A859B850E944A52181624F4C886D9861F
:10711000EA86FB86DF91CF91FF90EF90DF90CF90D2
:107120000895CF92DF92EF92FF920F931F9382E91F
:107130009BE065DF0E940F4D6093DD097093DE09CF
:107140008093DF099093E0092091920B3091930B8B
:107150004091940B5091950B6091BD0B7091BE0BBB
:107160008091BF0B9091C00B0E944750811179C054
:107170002091960B3091970B4091980B5091990B61
:107180006091C10B7091C20B8091C30B9091C40BA5
:107190000E944750811165C020E030E040E752E492
:1071A00060912A0270912B0280912C0290912D0205
:1071B0000E944E50B4EACB2EBBE0DB2E7B018C014B
:1071C0002EE93BE04AE95BE066E97BE082E99BE08F
:1071D0000E94C2238091920B9091930BA091940BEB
:1071E000B091950B8093BD0B9093BE0BA093BF0BFA
:1071F000B093C00B8091960B9091970BA091980B38
:10720000B091990B8093C10B9093C20BA093C30BC9
:10721000B093C40B80919A0B90919B0BA0919C0B07
:10722000B0919D0B8093C50B9093C60BA093C70B99
:10723000B093C80B80919E0B90919F0BA091A00BD7
:10724000B091A10B8093C90B9093CA0BA093CB0B69
:10725000B093CC0B1F910F91FF90EF90DF90CF90E8
:10726000089560913D0270913E02882777FD8095D8
:10727000982F0E94E95020912A0230912B024091D0
:107280002C0250912D020E941C5320E030E040E778
:1072900052E40E944E5020E030E048EC52E488CFA7
:1072A000AF92BF92CF92DF92EF92FF920F931F9314
:1072B000CF93DF93D82F20918A0B30918B0B409185
:1072C0008C0B50918D0B6091860B7091870B809188
:1072D000880B9091890B0E945752C62F172F082FA9
:1072E000F92E60913D0270913E02882777FD8095CE
:1072F000982F0E94E95020912A0230912B02409150
:107300002C0250912D020E941C5320E030E040E7F7
:1073100052E40E944E5020E030E048EC52E40E94DB
:107320004E502091A40B2F93DF93FF920F931F9346
:10733000CF935B016C01C2E0EC2E01E020E046E857
:107340005BE062E97BE08DEB9BE00E94042E809184
:10735000920B9091930BA091940BB091950B80930D
:10736000BD0B9093BE0BA093BF0BB093C00B80914D
:10737000960B9091970BA091980BB091990B8093DD
:10738000C10B9093C20BA093C30BB093C40B80911D
:107390009A0B90919B0BA0919C0BB0919D0B8093AD
:1073A000C50B9093C60BA093C70BB093C80B8091ED
:1073B0009E0B90919F0BA091A00BB091A10B80937D
:1073C000C90B9093CA0BA093CB0BB093CC0B0E942C
:1073D0000F4D6093DD097093DE098093DF09909370
:1073E000E0090F900F900F900F900F900F90DF918A
:1073F000CF911F910F91FF90EF90DF90CF90BF90B2
:10740000AF900895F8940E94B60D179A169A159A9F
:10741000149A60E084E00E94134EEDE8F1E184915B
:10742000882341F09091C00095FFFCCF8093C60067
:107430003196F5CFE5EFFDE08491882341F09091FE
:10744000C00095FFFCCF8093C6003196F5CF8091A8
:10745000C00085FFFCCF8AE08093C600FFCFCF92AB
:10746000DF92EF92FF920F931F930E940F4D0091B6
:10747000D9091091DA092091DB093091DC09C0901B
:10748000DD09D090DE09E090DF09F090E0096C1989
:107490007D098E099F09061717072807390728F461
:1074A000012B022B032B09F0ADDF80912602909176
:1074B0002702A0912802B0912902892B8A2B8B2BBD
:1074C00009F10E940F4D0091DD091091DE09209114
:1074D000DF093091E009601B710B820B930B009167
:1074E00026021091270220912802309129020617C6
:1074F00017072807390730F49091790480917804B0
:10750000981741F01F910F91FF90EF90DF90CF906F
:107510000C94A523179A169A159A149AF3CF0E94E1
:10752000B60D8091CF09811134C081E08093CF09DD
:107530008091760B9091770BA091780BB091790B9D
:107540008093720B9093730BA093740BB093750B95
:10755000EDE8F1E18491882341F09091C00095FF1E
:10756000FCCF8093C6003196F5CFEFE7FDE0849124
:10757000882341F09091C00095FFFCCF8093C60016
:107580003196F5CF8091C00085FFFCCF8AE08093D3
:10759000C60008958091CF090895CF93DF93EC0141
:1075A0008091A40B8093D00984E5BFD9811102C0DA
:1075B00080E064C0A6D90E94BB506093D0096623C6
:1075C000B9F3E7E8F1E18491882341F09091C0009C
:1075D00095FFFCCF8093C6003196F5CFC936D10513
:1075E00099F034F4C836D105C9F5E3E2F3E015C0EB
:1075F000CD36D10531F0CA3DD10581F5EEEDF2E091
:107600002AC0E5EFF2E01DC0ECE0F3E010C090917D
:10761000C00095FFFCCF8093C60081918111F7CF08
:107620001DC09091C00095FFFCCF8093C600819152
:107630008111F7CF13C09091C00095FFFCCF8093CC
:10764000C60081918111F7CF09C09091C00095FFCC
:10765000FCCF8093C60081918111F7CF40E050E0CC
:107660006091D00983ED9BE00E94044B8091C000A3
:1076700085FFFCCF8AE08093C60081E0DF91CF9147
:1076800008952F923F924F925F926F927F928F92C6
:107690009F92AF92BF92CF92DF92EF92FF920F93A1
:1076A0001F93CF93DF93CDB7DEB7A4970FB6F894AF
:1076B000DEBF0FBECDBF87E438D9882309F4FAC1F5
:1076C00020D90E94B65064307105B1F144F46230A3
:1076D000710511F144F577FF17C00C94DB476A354B
:1076E000710509F493C134F46C31710509F461C07A
:1076F0000C94DB476B35710509F48CC16C35710551
:1077000009F48DC10C94DB478091CF09811104C02D
:10771000C9DB07DD0C943B498091CF09811103C07F
:1077200040DC81E006C08091CF09811105C039DCC1
:1077300080E0B6DD0C943B4980E5F7D8882331F032
:10774000E0D80E94BB504B015C0103C0812C912CFE
:10775000540183E5EAD8882359F0D3D820E030E0FB
:107760004AE754E40E941C530E94BB504B015C0149
:107770000E94E91B0E940F4D6B017C01C80CD91CB3
:10778000EA1CFB1C0E940F4D6093DD097093DE091B
:107790008093DF099093E0090E940F4D6C157D05E1
:1077A0008E059F0510F00C94DB470E94340B57DECA
:1077B000F3CF80912A0290912B02A0912C02B091DC
:1077C0002D0280937E0B90937F0BA093800BB09340
:1077D000810B80913D0290913E029093CE0B80935D
:1077E000CD0B84E690E090933E0280933D020E9490
:1077F0000F4D6093DD097093DE098093DF0990934C
:10780000E00981E00E94A3148091BD0B9091BE0B12
:10781000A091BF0BB091C00B8093920B9093930BF0
:10782000A093940BB093950B8091C10B9091C20BD8
:10783000A091C30BB091C40B8093960B9093970BC0
:10784000A093980BB093990B8091C50B9091C60BA8
:10785000A091C70BB091C80B80939A0B90939B0B90
:10786000A0939C0BB0939D0B8091C90B9091CA0B78
:10787000A091CB0BB091CC0B80939E0B90939F0B60
:10788000A093A00BB093A10B10922A0210922B028E
:1078900010922C0210922D0288E547D8882311F00F
:1078A00090E008C089E541D88111FACF8AE53DD83A
:1078B00091E0982790932E0291110C94DE4788E571
:1078C00034D881110C94DE4780912E0281110C94E2
:1078D000E44789E52AD881110C94E44780912E026F
:1078E00081110C94EA478AE520D881110C94EA476B
:1078F00088E51BD88823C9F00DD8672B682B692B26
:10790000A1F00E9481342091B10B3091B20B4091D3
:10791000B30B5091B40B0E946E4F6093BD0B7093EC
:10792000BE0B8093BF0B9093C00B89E50E949534EA
:107930008823D1F00E948A34672B682B692BA1F031
:107940000E9481342091B50B3091B60B4091B70B5A
:107950005091B80B0E946E4F6093C10B7093C20B95
:107960008093C30B9093C40B8AE50E9495348823BF
:10797000D1F00E948A34672B682B692BA1F00E94FA
:1079800081342091B90B3091BA0B4091BB0B5091CF
:10799000BC0B0E946E4F6093C50B7093C60B809317
:1079A000C70B9093C80B29EC3BE045EC5BE061EC26
:1079B0007BE08DEB9BE00E943F2D80E00E94A314B2
:1079C00080917E0B90917F0BA091800BB091810BE9
:1079D00080932A0290932B02A0932C02B0932D0245
:1079E0008091CD0B9091CE0B90933E0280933D02FF
:1079F0000E940F4D6093DD097093DE098093DF09CB
:107A00009093E0090E949C140C94DB471092710B38
:107A10000C94DB4781E08093710B0C94DB4785E489
:107A20000E949534811102C00E94E91B94EDC92E79
:107A300093E0D92E21EBE22E2BE0F22E0DEB1BE092
:107A4000B12CD6018D916D010E949534882339F1B6
:107A5000B3E0BB120CC00E948134F80160837183D3
:107A60008283938389EC9BE00E94E42D18C00E94DE
:107A70008134D7012D913D914D915C910E946E4FC3
:107A8000F801608371838283938329EC3BE045ECAA
:107A90005BE061EC7BE08DEB9BE00E943F2DB394BB
:107AA000F4E0EF0EF11C0C5F1F4F24E0B212C9CFBF
:107AB0000C94DB478DE40E949534882311F40C94D8
:107AC00012470E9481340E94B6506837710509F44C
:107AD000B8C50CF07AC06535710509F432C47CF57F
:107AE0006035710509F4EEC3D4F46231710509F40F
:107AF000F6C35CF46131710511F00C94DB47179803
:107B00001698159814980C94DB476F31710509F499
:107B1000E9C06A32710509F468C10C94DB4762352B
:107B2000710509F4D5C30CF4D0C36335710509F4AC
:107B3000D2C36435710509F4D2C30C94DB476B36AC
:107B4000710509F4BAC324F56836710509F478C1E2
:107B5000ACF46C35710511F00C94DB4784ED93E0C7
:107B600098A38F8F0BEA19E06BEB862E69E0962EB7
:107B70007FE6A72E79E0B72E312C5AC469367105FD
:107B800009F48CC16A36710509F469C30C94DB47AA
:107B90006337710509F45EC464F46D36710509F448
:107BA0003AC26237710511F00C94DB47EFE7FEE053
:107BB00076C46537710509F45BC46737710511F048
:107BC0000C94DB47E9E4F3E046C56D3231E073071E
:107BD00009F42FC7D4F56B3C710509F455C6E4F4DC
:107BE0006C38710509F449C13CF46937710511F02D
:107BF0000C94DB4781E026C56E3B710509F48EC20B
:107C0000693C710511F00C94DB4754EDE52E53E00F
:107C1000F52E00E010E00BC66E3C710509F4CFC6EE
:107C200054F46C3C710509F44CC66D3C710509F4C3
:107C300068C60C94DB476C3D710509F4DCC66D3DEC
:107C4000710509F4E7C60C94DB47603991E07907C8
:107C500011F40C942C46A4F46F32B1E07B0709F4C4
:107C6000C3C70CF4BDC76E35F1E07F0711F40C9467
:107C700080466F35714011F40C94B6460C94DB4786
:107C80006B3833E0730709F4ECC75CF4653F91E0AF
:107C9000790709F4E4C7663F714009F4E0C70C9422
:107CA000DB476C38B3E07B0711F40C946546673E04
:107CB000734011F00C94DB471092CF098091720B46
:107CC0009091730BA091740BB091750B8093760B10
:107CD0009093770BA093780BB093790B0E94D034DC
:107CE0000C94DB470E940F4D6093D1097093D20929
:107CF0008093D3099093D4090091D5091091D609A6
:107D00002091D7093091D809601B710B820B930B1E
:107D100028EE33E040E050E00E940A54CA01B90165
:107D20002CE330E040E050E00E940A547F936F93D0
:107D30003F932F938CE49FE09F938F938E010F5F6F
:107D40001F4F1F930F930E946557E7E8F1E184915D
:107D50000FB6F894DEBF0FBECDBF882349F09091D7
:107D6000C00095FFFCCF8093C60031968491F5CF7B
:107D7000F8018191882339F09091C00095FFFCCFE4
:107D80008093C600F6CF8091C00085FFFCCF8AE0CB
:107D90008093C60080914A09882311F40C94DB4734
:107DA00010924A090091A40B10E0000F111F085D0A
:107DB0001B4FD8016D917C91882777FD8095982F76
:107DC0000E94E95020911E0230911F024091200232
:107DD000509121020E944A52181614F00C94DB476D
:107DE000F801118210820C94DB4783E50E949534E0
:107DF000882311F40C94DB470E9481346B017C01D1
:107E000080E50E949534882351F0C701B6010E9495
:107E1000B6506F3F710509F010F40C94F0476DE017
:107E200070E020E0E22FEE0FFF0BE456FC4F808164
:107E300091818617970711F40C94DB472F5FF2CFDF
:107E400088E690E0AADB81110C94DB4783E50E9471
:107E50009534882371F00091D0090E94813410E09C
:107E6000000F111F085D1B4F0E94B650D8016D9383
:107E70007C930E94B50D0C94DB4783E50E949534FA
:107E8000882311F40C94DB470E9481340E94B65081
:107E900070932704609326040C94DB4789E690E0F6
:107EA0007CDB81110C94DB47E6E4FFE084918823BE
:107EB00041F09091C00095FFFCCF8093C6003196B1
:107EC000F5CFE091D009B4E0EB9FF0011124E05E22
:107ED000FB4F408151816281738121E030E083ED6D
:107EE0009BE00E94994BE3E4FFE08491882341F0FA
:107EF0009091C00095FFFCCF8093C6003196F5CFDE
:107F0000E091D009F0E0EE0FFF1FE85DFB4F6081CC
:107F10007181882777FD8095982F0E94E950AB01E9
:107F2000BC0121E030E083ED9BE00E94994BEFE340
:107F3000FFE08491882341F09091C00095FFFCCF31
:107F40008093C6003196F5CF40911A0450911B04DE
:107F500060911C0470911D0421E030E083ED9BE0F2
:107F60000E94994BECE3FFE08491882341F09091CB
:107F7000C00095FFFCCF8093C6003196F5CF60918D
:107F8000260470912704882777FD8095982F0E94FA
:107F9000E950AB01BC0121E030E083ED9BE00E94A1
:107FA000994BE8E3FFE08491882341F09091C00071
:107FB00095FFFCCF8093C6003196F5CF8091D00914
:107FC00090E00E94290B4AE050E0BC0183ED9BE069
:107FD0000E94CD4AE3E3FFE08491882341F0909131
:107FE000C00095FFFCCF8093C6003196F5CF8FEF90
:107FF0009FEF0E94290B4AE050E0BC0183ED9BE01B
:108000000E94CD4A8091C00085FFFCCF8AE080931A
:10801000C6000C943B498DE690E0BFDA8111CBC7D6
:1080200010924A0983E50E949534882371F00091EB
:10803000D0090E94813410E0000F111F085D1B4F12
:108040000E94B650F8017183608383E50E949534E5
:10805000882351F00E94813460931E0270931F02A6
:10806000809320029093210282E40E949534882319
:1080700051F00E9481346093220270932302809316
:1080800024029093250286E40E949534882369F0A7
:108090000E94813460931A0270931B0280931C0229
:1080A00090931D0281E080934A090E94B50D0E94C1
:1080B0000F4D4B015C010091D00910E0F801EE0F6B
:1080C000FF1FE85DFB4F60817181882777FD8095F8
:1080D000982F0E94E9502B013C01F801EE0FFF1F81
:1080E000EE0FFF1FE05EFB4F80819181A281B38183
:1080F0008F8F98A3A9A3BAA3CC24CA94DC2C7601B1
:10810000E0E3FFE094919BA3ECE2FFE0A491ACA339
:10811000E8E2FFE024906AE0362EC7C783E50E94BC
:108120009534882341F00E9481340E94B6507093A8
:108130002704609326040E940F4D6B017C01E5E249
:10814000FFE01491E1E2FFE00491EDE1FFE0B49083
:10815000EAE0AE2E6091260470912704882777FD0F
:108160008095982F0E94E95020911A0430911B04A9
:1081700040911C0450911D040E944A52181614F09C
:108180000C9418490E940F4D6C197D098E099F09A6
:10819000693E73408105910508F45DC0E091A40B30
:1081A00024E0E29FF0011124E05EFB4F4081518109
:1081B00062817381812FE5E2FFE0882349F090918D
:1081C000C00095FFFCCF8093C60031968491F5CF17
:1081D00022E030E083ED9BE00E94994B802FE1E2AA
:1081E000FFE0882349F09091C00095FFFCCF809379
:1081F000C60031968491F5CF6091A40B70E04AE0FF
:1082000050E083ED9BE00E94CD4A8B2DEDE1FFE035
:10821000882349F09091C00095FFFCCF8093C60061
:1082200031968491F5CF40911A0450911B046091CE
:108230001C0470911D0421E030E083ED9BE00E945E
:10824000994B8091C00085FFFCCFA092C6000E9490
:108250000F4D6B017C010E94340B01D97BCF83E56C
:108260000E949534882311F10E94813420E030E08F
:10827000A9010E94475087FD0FC00E94813420E071
:1082800030E04FE753E40E944A52181644F00E942F
:1082900081340E94B65005C060E070E002C06FEF0C
:1082A00070E07093A30B6093A20B85C68FEF90E0F4
:1082B0009093A30B8093A20B7EC61092A30B1092F7
:1082C000A20B79C69D9AA59876C69D9AA59A73C663
:1082D0001092D20B70C681E08093D20B6CC683E5FE
:1082E0000E949534882399F00E94813420E030E088
:1082F0004AE754E40E941C530E94BB50609326023C
:1083000070932702809328029093290254C688E52F
:108310000E949534811196C789E50E949534811198
:1083200091C78AE50E94953481118CC785E40E942B
:108330009534811187C70E94E91B149A0E94501C32
:108340003AC683E50E9495340E94813420E030E0F3
:108350004AE754E40E941C530E94BB506093D90921
:108360007093DA098093DB099093DC0924C6B3E0AB
:108370003B1268C00E9481346B017C0120E030E038
:1083800040EA51E40E94475087FF3FC0A701960191
:10839000F80160817181828193810E944E502B018E
:1083A0003C019B01AC01609183097091840980912B
:1083B0008509909186090E941C53609383097093EC
:1083C00084098093850990938609A3019201D401C1
:1083D0006D917D918D919C910E941C53F40160835D
:1083E000718382839383D5016D917D918D919C9151
:1083F0000E94E750A30192010E941C530E94BB50AF
:10840000F5016083718382839383D801CD92DD92DD
:10841000ED92FC92139733940C5F1F4FF4E08F0E94
:10842000911C24E0A20EB11C34E0331609F4C3C53C
:10843000AF8DB8A18D91B8A3AF8F0E9495348823DA
:1084400051F395CF0E948134F80160837183828358
:108450009383E1CFE2E8FEE08491882309F4ABC581
:108460009091C00095FFFCCF8093C6003196F4CF69
:108470008091E1099091E2096AE270E005960E941C
:108480005A57009709F497C5FC013197108293C59C
:108490009091C00095FFFCCF8093C60031968491E7
:1084A0008111F6CF4091BD0B5091BE0B6091BF0B77
:1084B0007091C00B22E030E083ED9BE00E94994B6D
:1084C000ECE7FEE08491882341F09091C00095FF95
:1084D000FCCF8093C6003196F5CF4091C10B5091EF
:1084E000C20B6091C30B7091C40B22E030E083EDAE
:1084F0009BE00E94994BE9E7FEE08491882341F0DC
:108500009091C00095FFFCCF8093C6003196F5CFC7
:108510004091C50B5091C60B6091C70B7091C80B71
:1085200022E030E083ED9BE00E94994BE6E7FEE01D
:108530008491882341F09091C00095FFFCCF8093F7
:10854000C6003196F5CF4091C90B5091CA0B60918E
:10855000CB0B7091CC0B22E030E083ED9BE00E94CE
:10856000994BEBE6FEE08491882341F09091C000A6
:1085700095FFFCCF8093C6003196F5CF0E94421C38
:108580000E94E9502091AB093091AC094091AD09AE
:108590005091AE090E944E50AB01BC0122E030E088
:1085A00083ED9BE00E94994BE8E6FEE084918823EE
:1085B00041F09091C00095FFFCCF8093C6003196AA
:1085C000F5CF81E00E94421C0E94E9502091AF0942
:1085D0003091B0094091B1095091B2090E944E50BA
:1085E000AB01BC0122E030E083ED9BE00E94994B9F
:1085F000E5E6FEE08491882341F09091C00095FF6C
:10860000FCCF8093C6003196F5CF82E00E94421CD9
:108610000E94E9502091B3093091B4094091B50905
:108620005091B6090E944E50AB01BC0122E030E0EF
:1086300083ED9BE00E94994B8091C00085FFFCCFA9
:10864000B7C480E00E94A314B6C49091C00095FF07
:10865000FCCF8093C60081918111F7CF8091C0003B
:1086600085FFFCCF8AE08093C600EDE5FEE08491B3
:10867000882341F09091C00095FFFCCF8093C60005
:108680003196F5CF1E9903C0EAE3F3E009C0E4E4B4
:10869000F3E006C09091C00095FFFCCF8093C60028
:1086A00081918111F7CF8091C00085FFFCCF8AE0D6
:1086B0008093C600E5E5FEE08491882341F0909127
:1086C000C00095FFFCCF8093C6003196F5CF02998C
:1086D00003C0EAE3F3E009C0E4E4F3E006C09091EC
:1086E000C00095FFFCCF8093C60081918111F7CF28
:1086F0008091C00085FFFCCF8AE08093C600EDE446
:10870000FEE08491882341F09091C00095FFFCCF5A
:108710008093C6003196F5CF1D9903C0EAE3F3E0DC
:1087200009C0E4E4F3E006C09091C00095FFFCCFDF
:108730008093C60081918111F7CF8091C00085FFA1
:10874000FCCF8AE08093C600E5E4FEE084918823B4
:1087500041F09091C00095FFFCCF8093C600319608
:10876000F5CF019903C0EAE3F3E009C0E4E4F3E0E4
:1087700006C09091C00095FFFCCF8093C600819108
:108780008111F7CF8091C00085FFFCCF8AE08093F4
:10879000C600EDE3FEE08491882341F09091C00093
:1087A00095FFFCCF8093C6003196F5CF1C9903C08E
:1087B000EAE3F3E009C0E4E4F3E006C09091C0000E
:1087C00095FFFCCF8093C60081918111F7CF8091F6
:1087D000C00085FFFCCF8AE08093C600E5E3FEE0A1
:1087E0008491882341F09091C00095FFFCCF809345
:1087F000C6003196F5CF379903C0EAE3F3E009C02C
:10880000E4E4F3E006C09091C00095FFFCCF8093B4
:10881000C60081918111F7CF8091C00085FFFCCF08
:10882000C7C30C5F1F4F0031110509F4C4C3D70142
:108830008D917D010E949534882399F30E948134A3
:10884000F801E556F64F6F010E94BB50D6016D93BB
:108850007D938D939C9313970E948134F801E15985
:10886000F64F6F01F801E555F64F208131814281C5
:1088700053810E941C530E94BB50D6016D937D937F
:108880008D939C931397CDCF04ED13E04BEBE42E27
:1088900049E0F42EF80181918F010E9495348823DC
:1088A00041F00E948134D7016D937D938D939C9309
:1088B0001397B4E0EB0EF11CE3E0083D1E0751F7FF
:1088C0007AC383E50E949534882351F00E94813455
:1088D00060939309709394098093950990939609F6
:1088E00084E50E949534882309F465C30E9481348D
:1088F00060938F09709390098093910990939209E6
:108900005AC383E50E949534882351F00E94813434
:1089100060939709709398098093990990939A09A5
:1089200084E50E949534882351F00E94813460933D
:108930007F0970938009809381099093820982E472
:108940000E949534882361F00E9481340E94BB50BC
:108950006093CB097093CC098093CD099093CE0995
:1089600088E50E949534882351F00E9481346093F9
:108970008B0970938C0980938D0990938E098AE5F9
:108980000E949534882351F00E94813460938709B6
:10899000709388098093890990938A0985E40E94DD
:1089A0009534882309F407C30E94813460938309B6
:1089B000709384098093850990938609FCC204ED25
:1089C00013E031EBE32E3BE0F32ED8018D918D01C6
:1089D0000E949534882339F00E948134F701608326
:1089E000718382839383F4E0EF0EF11C23E0073D53
:1089F000120759F7E0C283E50E949534882309F4F1
:108A0000DAC20E9481340E94B65070933E02609395
:108A10003D02D1C283E50E949534882309F4CBC27C
:108A20000E9481340E94B65070933C0260933B02D6
:108A3000C2C280E50E949534882351F00E9481349F
:108A400060931102709312028093130290931402A8
:108A500089E40E949534882381F00E9481342DEBB3
:108A600037E346E05EE30E941C5360930D0270936F
:108A70000E0280930F029093100284E40E949534BA
:108A8000882381F00E9481342DEB37E346E05EE3DA
:108A90000E944E506093090270930A0280930B0269
:108AA00090930C0283E40E949534882351F00E9435
:108AB00081346093050270930602809307029093BD
:108AC00008020E94120BE4E6F3E08191882339F05A
:108AD0009091C00095FFFCCF8093C600F6CFE7E6EB
:108AE000F3E08191882339F09091C00095FFFCCF8D
:108AF0008093C600F6CF409111025091120260910E
:108B000013027091140222E030E083ED9BE011D655
:108B1000EBE6F3E08191882339F09091C00095FF56
:108B2000FCCF8093C600F6CF2DEB37E346E05EE343
:108B300060910D0270910E0280910F0290911002CF
:108B40000E944E50AB01BC0122E030E083ED9BE07F
:108B5000F0D5EFE6F3E08191882339F09091C000E1
:108B600095FFFCCF8093C600F6CF2DEB37E346E0B0
:108B70005EE36091090270910A0280910B0290916C
:108B80000C020E941C53AB01BC0122E030E083EDDB
:108B90009BE0CFD5E3E7F3E08191882339F0909112
:108BA000C00095FFFCCF8093C600F6CF2DEB37E3D6
:108BB00046E05EE360910502709106028091070233
:108BC000909108020E941C53AB01BC0122E030E0EE
:108BD00083ED9BE0AED58091C00085FFFCCFE8C15E
:108BE00081E00E94012EE7C185E40E94953488232C
:108BF00041F00E9481340E94B6508B0177FD0AC07B
:108C000002C000E010E0C12CD12C26E1E22E23E4CA
:108C1000F22E06C0C12CD12C9CE8E92E92E4F92E4C
:108C200083E50E949534882321F00E9481346B01F2
:108C30007C0183E40E949534882331F00E948134C2
:108C40000E94B6509B0102C025E030E0A801C70198
:108C5000B6010E94DE0DAFC10E94E91BACC16AD50E
:108C6000AAC184EDE82E83E0F82ED12CD7018D9196
:108C70007D010E949534882339F00E9481340E943E
:108C8000B6508D2D0E946E1CD394B5E0DB12EECF52
:108C900082E40E949534882339F00E9481340E9436
:108CA000B65084E00E946E1C83E50E9495348823B0
:108CB00061F0F12C0E9481340E94B6508F2D0E94E9
:108CC0006E1CF394E5E0FE12F5CF80E50E9495342A
:108CD000882329F00E9481340E94BB50162F83E51F
:108CE0000E949534882329F00E9481340E94BB5051
:108CF000062F602F70E0812F90E00E94561C5BC110
:108D000083E50E949534811104C004ED13E0F12C39
:108D100010C010E00E9481340E94BB50812F0E943D
:108D2000111D1F5F1530B1F7F0CFF394B5E0FB16BE
:108D300079F0D8018D918D010E9495348823A9F393
:108D40000E9481340E94BB508F2D0E94111DEDCFD7
:108D500082E40E949534882309F461C00E94813422
:108D60000E94BB5084E00E94111D59C083E50E94FF
:108D70009534882309F453C00E9481340E94B65070
:108D80006130710541F06230710509F048C004EDB1
:108D900013E0F12C25C004ED13E0F12CF8018191D2
:108DA0008F010E949534882341F00E9481340E94F3
:108DB000B6504FEF8F2D0E94C01CF394F5E0FF12C8
:108DC000EDCF82E40E949534882349F10E948134DA
:108DD0000E94B6504FEF20C0F394B5E0FB1689F027
:108DE000D8018D918D010E9495348823A9F30E94AA
:108DF00081340E94B650462F6FEF8F2D0E94C01C09
:108E0000EBCF82E40E949534882349F00E9481349C
:108E10000E94B650462F6FEF84E00E94C01C0E9453
:108E2000CC1DC9C084E50E949534882309F47FC015
:108E30000E9481340E94BB506093D009662389F15F
:108E4000E7E8F1E18491882341F09091C00095FF1B
:108E5000FCCF8093C6003196F5CFE7E7F3E0819130
:108E6000882339F09091C00095FFFCCF8093C60015
:108E7000F6CF40E050E06091D00983ED9BE0C4D391
:108E8000E9E7F3E08191882339F09091C00095FFE4
:108E9000FCCF8093C600F6CF8091C00085FFFCCF49
:108EA00087C086E40E9495348823D9F00E948134DB
:108EB0006B017C016093820B7093830B8093840B16
:108EC0009093850B20E030E0A9010E944A521816C9
:108ED00044F4C0922A02D0922B02E0922C02F0922B
:108EE0002D02E7E8F1E18491882341F09091C000E0
:108EF00095FFFCCF8093C6003196F5CFEAE8F3E00A
:108F00008191882339F09091C00095FFFCCF809328
:108F1000C600F6CF6091A40B70E04AE050E083ED0C
:108F20009BE03BD38091C00085FFFCCF41C0E7E8C8
:108F3000F1E18491882341F09091C00095FFFCCF2E
:108F40008093C6003196F5CFE2E2FEE0849188235B
:108F500041F09091C00095FFFCCF8093C600319600
:108F6000F5CF8091EB099091EC0920E6289FF00164
:108F7000299FF00D1124EF50F64F8191882339F08D
:108F80009091C00095FFFCCF8093C600F6CFE0E241
:108F9000FEE08491882341F09091C00095FFFCCFC2
:108FA0008093C6003196F5CF8091C00085FFFCCF3D
:108FB0008AE08093C6000E94B1345DC180E090E0F9
:108FC0000E941A310C94643C81E090E00E941A31B6
:108FD0000C946E3C82E090E00E941A310C94783C34
:108FE0000E9481340E94B6500C94113F18D58B0119
:108FF0009C01C701B601605F784D8F4F9F4F601B8A
:10900000710B820B930B28EE33E040E050E00E949E
:109010000A54BA01A9012AE030E083ED9BE0E9D2CD
:109020008091C00085FFFCCF3092C600F8D44B0180
:109030005C010E94340B0E942F3AEFEFCE16DE0641
:10904000EE06FE0609F0A8C02F8D38A149A15AA14D
:10905000C301B2010E944A52E091D009F0E08F01B1
:10906000000F111F000F111F005E1B4FEE0FFF1F9F
:10907000E85DFB4F6081718118160CF077C088277E
:1090800077FD8095982F0E94E95020E030E040E87D
:109090005FE323D79B01AC01D8016D917D918D9148
:1090A0009C910E944A5287FFB0C0B9D468197909CF
:1090B0008A099B09693E73408105910508F4B9CF7F
:1090C0008BA1E0E3FFE0882349F09091C00095FF79
:1090D000FCCF8093C60031968491F5CFE091D00902
:1090E000B4E0EB9FF0011124E05EFB4F4081518121
:1090F0006281738121E030E083ED9BE01AD38CA183
:10910000ECE2FFE0882349F09091C00095FFFCCF8E
:109110008093C60031968491F5CF6091D00970E0BC
:109120004AE050E083ED9BE038D2822DE8E2FFE098
:10913000882349F09091C00095FFFCCF8093C60032
:1091400031968491F5CFF7FE51CFE2E6F3E006C009
:109150009091C00095FFFCCF8093C6008191811152
:10916000F7CF8091C00085FFFCCF5ECF882777FDC9
:109170008095982F0E94E95020E030E040E85FE3BE
:10918000ADD69B01AC01F801608171818281938130
:109190007ED71816D4F589CFF7FC2DC0E091D00901
:1091A000F0E08F01000F111F000F111F005E1B4F19
:1091B000EE0FFF1FE85DFB4F60817181882777FD0F
:1091C0008095982F0E94E9509B01AC01D8016D91C8
:1091D0007D918D919C9181D6C9D797FF07C09095BD
:1091E0008095709561957F4F8F4F9F4F64307105CB
:1091F0008105910554F4F7FC12C011D46C197D0956
:109200006031774208F451CF0AC009D46B017C0168
:109210006F3FEFEF7E078E079E0769F746CFFFD3BC
:109220006093D5097093D6098093D7099093D80994
:10923000F6D36093DD097093DE098093DF09909384
:10924000E009B9CE0E94E91B88E50E94953481119E
:10925000179A89E50E9495348111169A8AE50E9431
:1092600095348111159A85E40E949534882309F478
:10927000A2CE149AA0CEA4960FB6F894DEBF0FBE6D
:10928000CDBFDF91CF911F910F91FF90EF90DF90B5
:10929000CF90BF90AF909F908F907F906F905F9096
:1092A0004F903F902F9008958091E7099091E809A1
:1092B000039714F40E94FB348091E7099091E80928
:1092C000892BC1F00E94413B8091E7099091E80908
:1092D00001979093E8098093E7098091EB099091B9
:1092E000EC09019664E070E00E94F7539093EC095A
:1092F0008093EB090E94340B0E942F3A0C940D14BA
:109300001F920F920FB60F9211240BB60F922F934C
:109310003F934F935F936F938F939F93EF93FF933D
:109320006091C6002091540C3091550CC9010196F2
:109330008F7799274091560C5091570C84179507B9
:1093400041F0F901EC52F44F60839093550C8093F7
:10935000540CFF91EF919F918F916F915F914F917D
:109360003F912F910F900BBE0F900FBE0F901F904B
:1093700018959A01AB01211581EE38074105510579
:1093800049F182E08093C00060E079E08DE390E0F5
:109390000E942C542150310941095109CA01B901D7
:1093A00022E030E040E050E00E942C543093C500B1
:1093B0002093C4008091C10080618093C10080919E
:1093C000C10088608093C1008091C1008068809353
:1093D000C10008951092C00020E130E0E7CF209155
:1093E000560C3091570C8091540C9091550C82176B
:1093F000930771F0F901EC52F44F80812F5F3F4FDA
:109400002F7733273093570C2093560C90E0089514
:109410008FEF9FEF08958091560C9091570C909389
:10942000550C8093540C08954F925F926F927F92E7
:109430008F929F92AF92BF92CF92DF92EF92FF9264
:109440000F931F93CF93DF93CDB7DEB7A0970FB6DF
:10945000F894DEBF0FBECDBF5C014115510561051B
:109460007105E9F420E030E040E350E060E070E0B6
:10947000A0960FB6F894DEBF0FBECDBFDF91CF919F
:109480001F910F91FF90EF90DF90CF90BF90AF9022
:109490009F908F907F906F905F904F905BC08E01F8
:1094A0000F5F1F4FC12CD12C76014801422E512C49
:1094B000612C712C8FEFC81AD80AE80AF80ACB0180
:1094C000BA01A30192010E940A54CA01F8016193F2
:1094D0008F01A901BC01411551056105710551F7C5
:1094E000F1E0CF1AD108E108F108F401EC0DFD1DFF
:1094F00080818A3010F440E301C047E3480F5527CC
:1095000047FD5095652F752F20E030E0C50122D032
:1095100081E0C81AD108E108F108EFEFCE16DE06A7
:10952000EE06FE0611F7A0960FB6F894DEBF0FBE4A
:10953000CDBFDF91CF911F910F91FF90EF90DF9002
:10954000CF90BF90AF909F908F907F906F905F90E3
:109550004F9008952115310539F48091C00085FFA1
:10956000FCCF4093C60008952A30310509F41CC091
:109570005BCFCF93DF93EC0120E030E04DE050E093
:1095800060E070E0E7DF20E030E04AE050E060E0DB
:1095900070E0CE01DF91CF91DDCF9A01AB0166275C
:1095A00057FD6095762FD6CFCF92DF92EF92FF9244
:1095B000CF93DF93EC016A017B0177FF0FC020E0BE
:1095C00030E04DE250E060E070E0C4DFF094E09401
:1095D000D094C094C11CD11CE11CF11C2AE0B7013D
:1095E000A601CE01DF91CF91FF90EF90DF90CF9059
:1095F0001BCF2115310539F48091C00085FFFCCFC8
:109600004093C600089510CF9A01462F50E060E0C5
:1096100070E0EFCFCF93DF93EC019A01AB0160E0F4
:1096200070E0E7DFCE01DF91CF91A3CF8F929F92C1
:10963000AF92BF92CF92DF92EF92FF921F93CF93A0
:10964000DF93EC016A017B01122F20E030E0A901D9
:10965000C701B6011CD587FF0CC020E030E04DE209
:1096600050E060E070E0CE0175DFF7FAF094F7F8B3
:10967000F094B12C60E070E080E09FE3B11639F027
:1096800020E030E040E251E409D5B394F7CF9B01EC
:10969000AC01C701B60122D46B017C016CD54B0132
:1096A0005C0195D59B01AC01C701B60116D46B01D5
:1096B0007C012AE0B501A401CE01B6DE112361F0E0
:1096C000E9ECF2E08191882339F09091C00095FF98
:1096D000FCCF8093C600F6CF1123F9F020E030E0F4
:1096E00040E251E4C701B601A7D76B017C013ED52A
:1096F0004B01AA2497FCA094BA2CB501A401CE0179
:1097000053DFC501B40165D59B01AC01C701B601AA
:10971000E4D36B017C011150DFCFDF91CF911F911A
:10972000FF90EF90DF90CF90BF90AF909F908F9081
:1097300008957CCFAF92BF92CF92DF92EF92FF92CB
:109740000F931F93CF93DF93CDB7DEB7E0970FB69C
:10975000F894DEBF0FBECDBF80E1EEE5F2E0DE01A2
:10976000919601900D928A95E1F780E1EEE6F2E0A4
:10977000DE01519601900D928A95E1F780E1EEE7C6
:10978000F2E0DE01119601900D928A95E1F76E01EB
:1097900081E2C80ED11C8BEAE82E89E0F82E8E01FA
:1097A0000F5E1F4F6BEB79E0AE014F5F5F4F9BE9A0
:1097B000A92E99E0B92E24E030E0F6018191919133
:1097C000A191B1916F01F70181939193A193B1930D
:1097D0007F01F80181919191A191B1918F01FB01DC
:1097E00081939193A193B193BF01FA0181919191DA
:1097F000A191B191AF01F50181939193A193B1939F
:109800005F012150310921153105B9F680E090E062
:10981000AAEFB3E48093930990939409A0939509D8
:10982000B093960980E090E8ABE3B5E480938F09AC
:1098300090939009A0939109B0939209109297097F
:10984000109298091092990910929A0980E29EE468
:10985000A0E0B0E08093CB099093CC09A093CD0910
:10986000B093CE0910927F0910928009109281095D
:109870001092820980E090E0A0EAB0E480938B0926
:1098800090938C09A0938D09B0938E094DEC5CECFC
:109890006CEC7EE3409387095093880960938909B3
:1098A00070938A098093830990938409A093850912
:1098B000B09386091092B90B1092BA0B1092BB0BA1
:1098C0001092BC0B1092B50B1092B60B1092B70B06
:1098D0001092B80B1092B10B1092B20B1092B30B06
:1098E0001092B40B8AE999E9A1EBB1E480931102DB
:1098F00090931202A0931302B093140285E894EFA0
:10990000A0E1BEE380930D0290930E02A0930F029C
:10991000B093100280E190E7A9E5B4E480930902D6
:1099200090930A02A0930B02B0930C0280E090E0A7
:10993000A0E8BFE38093050290930602A09307027C
:10994000B0930802E0960FB6F894DEBF0FBECDBF0D
:10995000DF91CF911F910F91FF90EF90DF90CF900B
:10996000BF90AF90089561E085E396D161E085E313
:109970005AD18CB580618CBD8CB580648CBD61E0A2
:1099800084E351D161E083E34EC11F920F920FB681
:109990000F9211242F933F938F939F93AF93BF9375
:1099A0008091590C90915A0CA0915B0CB0915C0C79
:1099B0003091580C23E0230F2D3720F40196A11D80
:1099C000B11D05C026E8230F0296A11DB11D2093ED
:1099D000580C8093590C90935A0CA0935B0CB09345
:1099E0005C0C80915D0C90915E0CA0915F0CB0912D
:1099F000600C0196A11DB11D80935D0C90935E0CCF
:109A0000A0935F0CB093600CBF91AF919F918F9129
:109A10003F912F910F900FBE0F901F9018952FB769
:109A2000F8946091590C70915A0C80915B0C909154
:109A30005C0C2FBF08953FB7F89480915D0C909116
:109A40005E0CA0915F0CB091600C26B5A89B05C080
:109A50002F3F19F00196A11DB11D3FBF6627782F3A
:109A6000892F9A2F620F711D811D911D42E0660F93
:109A7000771F881F991F4A95D1F70895CF92DF92DB
:109A8000EF92FF92CF93DF936B017C01D4DFEB0168
:109A9000C114D104E104F10471F0CDDF6C1B7D0B26
:109AA000683E7340A8F381E0C81AD108E108F108C4
:109AB000C851DC4FEDCFDF91CF91FF90EF90DF9059
:109AC000CF900895789484B5826084BD84B5816018
:109AD00084BD85B5826085BD85B5816085BDEEE6B6
:109AE000F0E0808181608083E1E8F0E01082808195
:109AF00082608083808181608083E0E8F0E0808103
:109B000081608083E1EBF0E0808184608083E0EB22
:109B1000F0E0808181608083E1E9F0E08081826013
:109B20008083808181608083E0E9F0E080818160D2
:109B30008083E1EAF0E080818260808380818160BF
:109B40008083E0EAF0E0808181608083E1E2F1E0FF
:109B5000808182608083808181608083E0E2F1E0A7
:109B6000808181608083EAE7F0E080818460808387
:109B70008081826080838081816080838081806831
:109B800080831092C100089590E0FC013197E1318B
:109B9000F10508F047C0E658FF4F7AC68091800073
:109BA0008F7703C0809180008F7D8093800008951F
:109BB00084B58F7702C084B58F7D84BD0895809170
:109BC000B0008F7703C08091B0008F7D8093B0008C
:109BD0000895809190008F7707C0809190008F7DCD
:109BE00003C080919000877F8093900008958091BA
:109BF000A0008F7707C08091A0008F7D03C0809167
:109C0000A000877F8093A0000895809120018F7726
:109C100007C0809120018F7D03C080912001877F44
:109C2000809320010895CF93DF9390E0FC01E652EA
:109C3000FE4E2491FC01E05EFD4E8491882349F1A3
:109C400090E0880F991FFC01E656FD4EA591B49156
:109C500080589D4EFC01C591D4919FB7611108C0F9
:109C6000F8948C91209582238C93888182230AC05A
:109C7000623051F4F8948C91322F309583238C9379
:109C80008881822B888304C0F8948C91822B8C93DA
:109C90009FBFDF91CF9108950F931F93CF93DF93D1
:109CA0001F92CDB7DEB7282F30E0F901EC56FE4EFB
:109CB0008491F901E652FE4E1491F901E05EFD4EE9
:109CC00004910023C1F0882319F069835DDF698165
:109CD000E02FF0E0EE0FFF1FE058FD4EA591B4918C
:109CE0009FB7F8948C91611103C01095812301C036
:109CF000812B8C939FBF0F90DF91CF911F910F917C
:109D00000895CF93DF93282F30E0F901EC56FE4EF3
:109D10008491F901E652FE4ED491F901E05EFD4EC8
:109D2000C491CC2389F081112FDFEC2FF0E0EE0FEE
:109D3000FF1FEA59FD4EA591B4912C912D2381E08E
:109D400090E021F480E002C080E090E0DF91CF91CC
:109D500008951F93CF93DF93182FEB0161E063DF2A
:109D6000209711F460E004C0CF3FD10531F461E0E9
:109D7000812FDF91CF911F918FCFE12FF0E0EC5633
:109D8000FE4E449150E0FA013197E131F10508F0BF
:109D900090C0E557FF4F7CC584B5806884BDC7BDC2
:109DA0008DC084B5806284BDC8BD88C080918000AC
:109DB000806880938000D0938900C09388007EC023
:109DC00080918000806280938000D0938B00C0934C
:109DD0008A0074C08091B00080688093B000C09306
:109DE000B3006CC08091B00080628093B000C093DB
:109DF000B40064C080919000806880939000D093FC
:109E00009900C09398005AC080919000806280931E
:109E10009000D0939B00C0939A0050C08091900016
:109E2000886080939000D0939D00C0939C0046C0B2
:109E30008091A00080688093A0008091A0008F7B1B
:109E40008093A000D093A900C093A80037C0809150
:109E5000A00080628093A000D093AB00C093AA00C2
:109E60002DC08091A00088608093A000D093AD00A9
:109E7000C093AC0023C080912001806880932001B2
:109E8000D0932901C093280119C0809120018062DC
:109E900080932001D0932B01C0932A010FC08091A1
:109EA0002001886080932001D0932D01C0932C0164
:109EB00005C0C038D1050CF05ACF54CFDF91CF91F7
:109EC0001F910895FFDD0E94C332C0E0D0E0ECD9BD
:109ED0002097E9F30E940000FACF5058BB27AA2729
:109EE0000ED076C23FD230F044D220F031F49F3F02
:109EF00011F41EF40FC20EF4E095E7FBDCC1E92F6C
:109F000089D280F3BA17620773078407950718F0A0
:109F100071F49EF5B8C20EF4E0950B2EBA2FA02D69
:109F20000B01B90190010C01CA01A0011124FF2706
:109F3000591B99F0593F50F4503E68F11A16F04001
:109F4000A22F232F342F4427585FF3CF4695379500
:109F50002795A795F0405395C9F77EF41F16BA0BC5
:109F6000620B730B840BBAF09150A1F0FF0FBB1F73
:109F7000661F771F881FC2F70EC0BA0F621F731FBC
:109F8000841F48F4879577956795B795F7959E3F19
:109F900008F0B3CF9395880F08F09927EE0F9795A7
:109FA00087950895DFD158F080E891E009F49EEF9D
:109FB000E0D128F040E851E059F45EEF09C0AAC1B1
:109FC00062C2E92FE07826D268F3092E052AC1F390
:109FD000261737074807590738F00E2E07F8E025EF
:109FE00069F0E025E0640AC0EF6307F8009407FA1F
:109FF000DB01B9019D01DC01CA01AD01EF935DD028
:10A00000E7D10AD05F91552331F02BED3FE049E4D1
:10A0100050FD49EC63CF0895DF93DD27B92FBF775B
:10A0200040E85FE31616170648075B0710F4D92FC0
:10A0300096D29F938F937F936F93A9D3E8E3F1E038
:10A040006CD1C6D12F913F914F915F9101D3DD2308
:10A0500049F09058A2EA2AED3FE049EC5FE3D0785E
:10A060005D274DDFDF91B4C1F7D180F09F3740F419
:10A0700091110EF409C260E070E080E89FE308955A
:10A0800026F01B16611D711D811D1BC135C1EFD04E
:10A0900008F481E0089575D1E395ABC10CD098C167
:10A0A00068D140F05FD130F021F45F3F19F003C177
:10A0B0005111EAC12FC1AED198F39923C9F35523A9
:10A0C000B1F3951B550BBB27AA27621773078407AB
:10A0D00038F09F5F5F4F220F331F441FAA1FA9F361
:10A0E00033D00E2E3AF0E0E830D091505040E69553
:10A0F000001CCAF729D0FE2F27D0660F771F881FB4
:10A10000BB1F261737074807AB07B0E809F0BB0BA2
:10A11000802DBF01FF2793585F4F2AF09E3F5105C6
:10A1200068F0C9C0B1C15F3FECF3983EDCF386959F
:10A1300077956795B795F7959F5FC9F7880F911D3C
:10A140009695879597F90895E1E0660F771F881F28
:10A15000BB1F621773078407BA0720F0621B730BDB
:10A16000840BBA0BEE1F88F7E095089504D068942D
:10A17000B1118AC1089556D188F09F5790F0B92F38
:10A180009927B751A0F0D1F0660F771F881F991F4C
:10A190001AF0BA95C9F712C0B13081F074D1B1E0AC
:10A1A000089571C1672F782F8827B85F39F0B93FBC
:10A1B000CCF3869577956795B395D9F73EF490954E
:10A1C0008095709561957F4F8F4F9F4F0895E894CC
:10A1D00009C097FB3EF490958095709561957F4FEF
:10A1E0008F4F9F4F9923A9F0F92F96E9BB2793959D
:10A1F000F695879577956795B795F111F8CFFAF4AD
:10A20000BB0F11F460FF1BC06F5F7F4F8F4F9F4FDD
:10A2100016C0882311F096E911C0772321F09EE83B
:10A22000872F762F05C0662371F096E8862F70E0A1
:10A2300060E02AF09A95660F771F881FDAF7880F7B
:10A240009695879597F9089507D180F09F3740F448
:10A2500091110EF019C160E070E080E89FEB089565
:10A2600026F41B16611D711D811D2BC045C0990F61
:10A270000008550FAA0BE0E8FEEF16161706E807D0
:10A28000F907C0F012161306E407F50798F0621BF1
:10A29000730B840B950B39F40A2661F0232B242BC6
:10A2A000252B21F408950A2609F4A140A6958FEFE5
:10A2B000811D811D089597F99F6780E870E060E037
:10A2C0000895882371F4772321F09850872B762FF7
:10A2D00007C0662311F499270DC09051862B70E0BA
:10A2E00060E02AF09A95660F771F881FDAF7880FCB
:10A2F0009695879597F908959F3F31F0915020F4F6
:10A30000879577956795B795880F911D9695879551
:10A3100097F908959FEF80EC0895DF93CF931F93F3
:10A320000F93FF92EF92DF927B018C01689405C03E
:10A33000DA2EEF018DD1FE01E894A591259135919A
:10A3400045915591AEF3EF01DADDFE019701A801C9
:10A35000DA9479F7DF90EF90FF900F911F91CF91F2
:10A36000DF91089500240A941616170618060906A8
:10A37000089500240A94121613061406050608957B
:10A38000C9CF50D0E8F3E894E0E0BB279F57F0F046
:10A390002AED3FE049EC06C0EE0FBB0F661F771FAA
:10A3A000881F28F0B23A62077307840728F0B25A70
:10A3B000620B730B840BE3959A9572F7803830F437
:10A3C0009A95BB0F661F771F881FD2F7904896CFCC
:10A3D000092E0394000C11F4882352F0BB0F40F4B3
:10A3E000BF2B11F460FF04C06F5F7F4F8F4F9F4FF3
:10A3F0000895EF93E0FF06C0A2EA2AED3FE049ECA2
:10A400005FEB7DDDE5DF0F90039401FC9058E5E6FE
:10A41000F1E0C7C157FD9058440F551F59F05F3FF9
:10A4200071F04795880F97FB991F61F09F3F79F076
:10A4300087950895121613061406551FF2CF4695F8
:10A44000F1DF08C0161617061806991FF1CF86957A
:10A450007105610508940895E5DFA0F0BEE7B9171E
:10A4600088F4BB279F3860F41616B11D672F782F2C
:10A470008827985FF7CF869577956795B11D939557
:10A480009639C8F30895E894BB2766277727CB0150
:10A4900097F90895ECDE08F48FEF089563DF19F063
:10A4A00068DF09F037CF07CFB901CA0125CF9F7701
:10A4B0005F77B0DF98F39923B9F35523B9F3FF27FA
:10A4C000951758F4E52FE91BED3070F75E3B10F05F
:10A4D000F1E41CC09034E0F40AC0E92FE51BED3034
:10A4E00028F79E3B10F0F1E411C0503488F4F9EAEB
:10A4F00088232AF09A95660F771F881FDAF744237E
:10A500002AF05A95220F331F441FDAF79F1B5F1B57
:10A51000FF931F930F93FF92EF9279018A01BB275C
:10A52000AB2F9B01AC0196D09701A801BF937B0193
:10A530008C01AA27BA2FB901CA018CD0AF9197011B
:10A54000A801EF90FF900F911F91D9DC41DFE1D07E
:10A550004F9140FF0895552747FD509509C09B0135
:10A56000AC0160E070E080E89FE398CDA4CEC4CE5B
:10A5700059DFE8F39923D9F3940F511DBBF39150A0
:10A58000504094F059F0882332F0660F771F881FEF
:10A5900091505040C1F79E3F510544F7880F911DDF
:10A5A0009695879597F908955F3FACF0983E9CF09B
:10A5B000BB27869577956795B79508F4B160939515
:10A5C000C1F7BB0F58F711F460FFE8CF6F5F7F4F03
:10A5D0008F4F9F4FE3CF58CF25DF58F19E5758F14B
:10A5E0009851A0F0E9F0983020F5092E9927660FD0
:10A5F000771F881F991F0A94D1F712C0062E672F64
:10A60000782F8827985F11F4000C07C0993FB4F3A6
:10A610008695779567959395D9F7611D711D811D75
:10A620003EF490958095709561957F4F8F4F9F4F29
:10A630000895689429CF27CF0BD0CACE93DE28F097
:10A6400098DE18F0952309F036CE64CE11241CCF85
:10A65000E1DEA0F3959FD1F3950F50E0551F629F67
:10A66000F001729FBB27F00DB11D639FAA27F00D6B
:10A67000B11DAA1F649F6627B00DA11D661F829F92
:10A680002227B00DA11D621F739FB00DA11D621F77
:10A69000839FA00D611D221F749F3327A00D611D94
:10A6A000231F849F600D211D822F762F6A2F112476
:10A6B0009F5750408AF0E1F088234AF0EE0FFF1FC9
:10A6C000BB1F661F771F881F91505040A9F79E3F00
:10A6D000510570F0F0CDD8CE5F3FECF3983EDCF33F
:10A6E000869577956795B795F795E7959F5FC1F73D
:10A6F000FE2B880F911D9695879597F908959F9346
:10A7000040DE0F9007FCEE5F74CE11F40EF402CE23
:10A71000F3CD88DED0F39923D9F3CEF39F57550BB1
:10A7200087FF38D00024A0E640EA90018058569573
:10A73000979528F4805C660F771F881F20F02617F6
:10A740003707480730F4621B730B840B202931292B
:10A750004A2BA69517940794202531254A2758F7A8
:10A76000660F771F881F20F026173707480730F439
:10A77000620B730B840B200D311D411DA09581F7D9
:10A78000B901842F9158880F9695879508959B015C
:10A79000AC0152CF91505040660F771F881FD2F7FF
:10A7A00008959F938F937F936F93FF93EF939B01F4
:10A7B000AC0142DFEF91FF91B0DD2F913F914F91BE
:10A7C0005F913ACFB7FF6AC069D0821B930B08959F
:10A7D000DB018F939F9362D0BF91AF91A29F800DB9
:10A7E000911DA39F900DB29F900D1124089597FB8A
:10A7F000072E16F4009406D077FD08D059D007FC38
:10A8000005D03EF4909581959F4F08957095619580
:10A810007F4F0895A1E21A2EAA1BBB1BFD010DC09C
:10A82000AA1FBB1FEE1FFF1FA217B307E407F50700
:10A8300020F0A21BB30BE40BF50B661F771F881FDC
:10A84000991F1A9469F760957095809590959B0172
:10A85000AC01BD01CF010895052E97FB16F40094BD
:10A860000FD057FD05D0D6DF07FC02D046F408C054
:10A8700050954095309521953F4F4F4F5F4F08952C
:10A8800090958095709561957F4F8F4F9F4F08955C
:10A89000EE0FFF1F0590F491E02D19941DD0A59F98
:10A8A000900DB49F900DA49F800D911D11240895CB
:10A8B000AA1BBB1B51E107C0AA1FBB1FA617B707E6
:10A8C00010F0A61BB70B881F991F5A95A9F7809502
:10A8D0009095BC01CD010895A29FB001B39FC00126
:10A8E000A39F700D811D1124911DB29F700D811DBC
:10A8F0001124911D08954F925F926F927F928F92D3
:10A900009F92AF92BF92CF92DF92EF92FF920F93FE
:10A910001F93CF93DF938B016115710521F0DB014C
:10A920008C9311969C93EC015E01BFEFAB1ABB0AAE
:10A930007501C8808C2D90E083D2892B11F0E50140
:10A94000F3CFEDE2CE1208C07E01F2E0EF0EF11C73
:10A95000C980DD24D39409C02BE2C21205C07E0158
:10A9600042E0E40EF11CC980D12CE701219743E0BD
:10A9700050E06CEB72E1CE016BD2892BC9F4E70198
:10A98000229645E050E067EB72E1CE0161D2892B5F
:10A9900011F4E70127960115110519F0D801CD939F
:10A9A000DC93D11002C160E070E080E89FE706C14F
:10A9B00043E050E064EB72E1CE014AD2892B59F4B6
:10A9C0000115110509F4F6C0B2E0EB0EF11CF80117
:10A9D000F182E082EFC0F70160E070E0CB01C0E0FF
:10A9E000D0E07F01A0EDAA2EAC0C29E02A1528F1B9
:10A9F0004D2D4260B42E2D2D2870D2FE04C02111A1
:10AA000024C0219622C021112197A5E0B0E09B012E
:10AA1000AC0144DF660F771F881F991F6A0D711DF7
:10AA2000811D911D6839A9E97A078A07A9E19A076A
:10AA300060F0BD2DB660BB2E08C02EEFA2120AC07A
:10AA4000D3FC50C04D2D4860B42E3196D701CC9028
:10AA5000DB2CC7CF2C2D2F7D253409F043C0A081DE
:10AA6000AD3241F4BD2DB061DB2E7F0122E0E20E5C
:10AA7000F11C0CC07F01AB3231F04FEFE41AF40A45
:10AA800021E030E006C0A2E0EA0EF11CA18122E044
:10AA900030E0A053AA3018F0E21AF30A23C0F701FD
:10AAA00020E030E02038BCE03B075CF4A901440F13
:10AAB000551F440F551F240F351F220F331F2A0F18
:10AAC000311DAF014F5F5F4F7A01A081A053AA30C3
:10AAD00010F4FA01E7CFD4FE03C031952195310976
:10AAE000C20FD31FD1FE09C00115110531F0E1E0FD
:10AAF000EE1AF108D801ED92FC9269DB2D2D23703E
:10AB0000233019F06B017C0106C06B017C01F7FA60
:10AB1000F094F7F8F09420E030E0A901C701B60105
:10AB2000B6DA882309F43EC0D7FF06C0D195C19597
:10AB3000D10903ED12E102C00BEE12E14801B8E1C8
:10AB40008B1A910890E2A92EB12CF80145905590EE
:10AB500065907490CA15DB0554F0A3019201C701FA
:10AB6000B6016ADD6B017C01CA19DB09F3CF045021
:10AB70001109B594A7940815190539F78E2D880F7A
:10AB80008F2D881F8F3F41F020E030E0A901C701E1
:10AB9000B6017DDA811106C082E290E09093660CE6
:10ABA0008093650CC701B60109C060E070E080E8E1
:10ABB0009FEF04C060E070E080EC9FE7DF91CF91F1
:10ABC0001F910F91FF90EF90DF90CF90BF90AF90CB
:10ABD0009F908F907F906F905F904F9008952F92ED
:10ABE0003F925F926F927F928F929F92AF92BF92AD
:10ABF000CF92DF92EF92FF920F931F93CF93DF9349
:10AC00008B01EA016115710521F0DB018C9311962E
:10AC10009C93209739F09E0122503109233231054F
:10AC200008F0F8C07C016701BFEFCB1ADB0A5601C0
:10AC3000F7016080862D90E003D1892B11F0760119
:10AC4000F2CFFDE26F120AC0570182E0A80EB11CDC
:10AC5000D70111966C90772473940BC0BBE26B12F2
:10AC600007C05701E2E0AE0EB11CD70111966C90FF
:10AC7000712CCE018F7E892B89F4B0E36B1222C038
:10AC8000F50180818F7D883541F56180F2E0AF0E5E
:10AC9000B11C872D8260782EC0E1D0E0C830D1058C
:10ACA000F1F04CF4C230D10511F5C12CD12CE12CBE
:10ACB000B0E4FB2E2EC0CA30D10531F0C031D10531
:10ACC00019F115C0209751F7CAE0D0E0ACECCA2EBC
:10ACD000DC2CEC2CACE0FA2E1CC02097F9F6C8E076
:10ACE000D0E0C12CD12CE12CF0E1FF2E12C060E0AD
:10ACF00070E080E090E89E01442737FD4095542F96
:10AD000089DD69017A0105C0C12CD12CE12CE8E074
:10AD1000FE2EF50160E020E030E0A9014E01AA24FA
:10AD200097FCA094BA2C1F0170ED572E560CA9E089
:10AD3000A51570F48FEB860D8A3118F499EC592E15
:10AD400006C08FE9860D8A3128F589EA582E560CFF
:10AD5000852D90E08C179D07ECF467FD17C0C21697
:10AD6000D306E406F50678F0C501B40131DD9B0198
:10AD7000AC01250D311D411D511D2130310541050D
:10AD8000B0E85B0710F06FEF01C061E03196D101D0
:10AD90006C90C9CF872D81700115110571F0662364
:10ADA00029F03197D801ED93FC9307C071FE19C0CB
:10ADB0003297D801ED93FC9314C067FF12C088232B
:10ADC00029F020E030E040E050E804C02FEF3FEFF2
:10ADD0004FEF5FE782E290E09093660C8093650C02
:10ADE00016C0882341F050954095309521953F4FEE
:10ADF0004F4F5F4F0CC057FF0AC082E290E0909324
:10AE0000660C8093650C2FEF3FEF4FEF5FE7B901C2
:10AE1000CA0104C060E070E080E090E0DF91CF9173
:10AE20001F910F91FF90EF90DF90CF90BF90AF9068
:10AE30009F908F907F906F905F903F902F9008959C
:10AE400091115FC2803219F089508550D0F7089572
:10AE5000FB01DC014150504088F08D9181341CF0A1
:10AE60008B350CF4805E659161341CF06B350CF40D
:10AE7000605E861B611171F3990B0895881BFCCFEE
:10AE8000FB0155915523A9F0BF01DC014D914517F8
:10AE90004111E1F759F4CD010590002049F04D91A1
:10AEA00040154111C9F3FB014111EFCF81E090E062
:10AEB00001970895FC018191861721F08823D9F725
:10AEC000992708953197CF0108950F931F93CF933A
:10AED000DF93CDB7DEB72E970FB6F894DEBF0FBE67
:10AEE000CDBF0E891F898EE08C831A8309838FEF73
:10AEF0009FE79E838D83AE01465E5F4F688D798D9F
:10AF0000CE01019610D0EF81F885E00FF11F10827D
:10AF10002E960FB6F894DEBF0FBECDBFDF91CF9156
:10AF20001F910F9108952F923F924F925F926F92CF
:10AF30007F928F929F92AF92BF92CF92DF92EF92C9
:10AF4000FF920F931F93CF93DF93CDB7DEB72C976C
:10AF50000FB6F894DEBF0FBECDBF7C016B018A0136
:10AF6000FC0117821682838181FFB0C1CE01019658
:10AF70004C01F7019381F60193FD859193FF819137
:10AF80006F01882309F49EC1853239F493FD8591C0
:10AF900093FF81916F01853221F4B70190E0CAD10E
:10AFA000E8CF512C312C20E02032A0F48B3269F014
:10AFB00030F4803259F0833269F420612CC08D3234
:10AFC00039F0803339F4216026C02260246023C028
:10AFD000286021C027FD27C030ED380F3A3078F4C3
:10AFE00026FF06C0FAE05F9E300D1124532E13C0D9
:10AFF0008AE0389E300D1124332E20620CC08E3230
:10B0000021F426FD5FC1206406C08C3611F420684F
:10B0100002C0883641F4F60193FD859193FF81913A
:10B020006F018111C1CF982F9F7D9554933028F4E3
:10B030000C5F1F4FFFE3F9830DC0833631F0833778
:10B0400071F0833509F057C021C0F80180818983F0
:10B050000E5F1F4F44244394512C540114C03801F7
:10B06000F2E06F0E711CF801A080B18026FF03C0D2
:10B07000652D70E002C06FEF7FEFC5012C874FD1C7
:10B080002C0183012C852F77222E16C03801F2E087
:10B090006F0E711CF801A080B18026FF03C0652DE2
:10B0A00070E002C06FEF7FEFC5012C872DD12C011E
:10B0B0002C852068222E830123FC19C0832D90E06B
:10B0C00048165906A0F4B70180E290E033D13A94D3
:10B0D000F5CFF50127FC859127FE81915F01B7012E
:10B0E00090E028D131103A94F1E04F1A5108411400
:10B0F000510479F7DEC0843611F0893631F5F80154
:10B1000027FF07C060817181828193810C5F1F4F8F
:10B1100008C060817181882777FD8095982F0E5F28
:10B120001F4F2F76B22E97FF09C09095809570958E
:10B1300061957F4F8F4F9F4F2068B22E2AE030E0FD
:10B14000A4012AD1A82EA81843C0853729F42F7E40
:10B15000B22E2AE030E025C0F22FF97FBF2E8F36C5
:10B16000C1F018F4883579F0ADC0803719F0883710
:10B1700021F0A8C02F2F2061B22EB4FE0DC08B2D60
:10B180008460B82E09C024FF0AC09F2F9660B92E94
:10B1900006C028E030E005C020E130E002C020E138
:10B1A00032E0F801B7FE07C060817181828193812E
:10B1B0000C5F1F4F06C06081718180E090E00E5FE0
:10B1C0001F4FA401E9D0A82EA818FB2DFF77BF2E92
:10B1D000B6FE0BC02B2D2E7FA51450F4B4FE0AC072
:10B1E000B2FC08C02B2D2E7E05C07A2C2B2D03C05F
:10B1F0007A2C01C0752C24FF0DC0FE01EA0DF11D53
:10B200008081803311F4297E09C022FF06C0739427
:10B21000739404C0822F867809F0739423FD12C0C2
:10B2200020FF06C05A2C731418F4530C5718732CB3
:10B23000731460F4B70180E290E02C877BD07394A4
:10B240002C85F6CF731410F4371801C0312C24FF6D
:10B2500011C0B70180E390E02C876CD02C8522FFD1
:10B2600016C021FF03C088E590E002C088E790E0A7
:10B27000B7010CC0822F867851F021FD02C080E218
:10B2800001C08BE227FD8DE2B70190E053D0A514F9
:10B2900030F4B70180E390E04DD05A94F8CFAA94EF
:10B2A000F401EA0DF11D8081B70190E043D0A110B7
:10B2B000F6CF332009F45DCEB70180E290E03AD0BA
:10B2C0003A94F7CFF7018681978102C08FEF9FEF05
:10B2D0002C960FB6F894DEBF0FBECDBFDF91CF9195
:10B2E0001F910F91FF90EF90DF90CF90BF90AF90A4
:10B2F0009F908F907F906F905F904F903F902F9096
:10B300000895992788270895FC01059061507040A1
:10B310000110D8F7809590958E0F9F1F0895FC011E
:10B320006150704001900110D8F7809590958E0F74
:10B330009F1F08950F931F93CF93DF93182F092F0B
:10B34000EB018B8181FD03C08FEF9FEF20C082FF57
:10B3500010C04E815F812C813D81421753077CF4E0
:10B36000E881F9819F012F5F3F4F39832883108344
:10B3700006C0E885F985812F1995892B29F72E813B
:10B380003F812F5F3F4F3F832E83812F902FDF918F
:10B39000CF911F910F910895FA01AA27283051F1FA
:10B3A000203181F1E8946F936E7F6E5F7F4F8F4FF6
:10B3B0009F4FAF4FB1E03ED0B4E03CD0670F781F55
:10B3C000891F9A1FA11D680F791F8A1F911DA11D3A
:10B3D0006A0F711D811D911DA11D20D009F4689473
:10B3E0003F912AE0269F11243019305D3193DEF61B
:10B3F000CF010895462F4770405D4193B3E00FD0D1
:10B40000C9F7F6CF462F4F70405D4A3318F0495DBB
:10B4100031FD4052419302D0A9F7EACFB4E0A6959E
:10B420009795879577956795BA95C9F700976105C0
:10B43000710508959B01AC010A2E06945795479516
:10B4400037952795BA95C9F7620F731F841F951F0B
:08B45000A01D0895F894FFCF40
:10B4580001FF3FFF3F0000803F1070594485F41002
:10B468003E9A99B1410101010101CDCCCC3D0000CA
:10B47800524300007A4360EA00000080BB440100A8
:10B488000095430080894300007A4364006400000B
:10B49800803B4500803B45000070430000000004ED
:10B4A80005030001A5A5DC87871010041010000013
:10B4B800C9420000C9420000484400004844000056
:10B4C800FA430000FA4300002041000034422823D8
:10B4D80000002823000064000000102700005049E5
:10B4E80044204175746F74756E652073746172744D
:10B4F80000504944204175746F74756E652066610B
:10B50800696C65642E204261642065787472756484
:10B518006572206E756D6265722E00537465707267
:10B5280061746520746F20686967683A20004D323D
:10B53800313820496E76616C69642065787472755B
:10B5480064657220004D31303920496E76616C692E
:10B558006420657874727564657220004D313035E9
:10B5680020496E76616C69642065787472756465CB
:10B578007220004D31303420496E76616C69642048
:10B58800657874727564657220005452494747455E
:10B59800524544006F70656E005265706F72746931
:10B5A8006E6720656E6473746F7020737461747550
:10B5B80073003F006F6B0020703A0020693A00204A
:10B5C800643A0020633A005400496E76616C6964FD
:10B5D8002065787472756465720041637469766574
:10B5E8002045787472756465723A20000000010085
:10B5F800250030001D000C001800240031001C003C
:10B608000B00170023002F001B000A001E00040077
:10B618000300080022002B001A000900360037003A
:08B628003500380058595A455D
:00000001FF
